:107410000000050200000301FA0400EF0500030A62
:107420000A5A0B001E0C00FA0D00030E00040F0197
:1074300064100096120132130AFA14010217010AAD
:107440001801EF1905321A010A1B01EF1C05321F42
:10745000FFFF20FFFF23011E2400642A00FA2B00F7
:10746000FA2C50782D003D2E0046300064325078C2
:107470003300003432FA3501643601643701503884
:107480000A643A00033B00043C00643E003C3F00B9
:107490000140FFFF411450420A5A430AC8440532D2
:1074A0004500B44600FA4900024B00014C00FA5076
:1074B0000606510596520A32530B46540A96570552
:1074C00046590A465A32FA5B010A5C0A325E000AE1
:1074D0005F00646200FE64021C67FFFF68010169CF
:1074E00001016A05966B00006C32966D0004730012
:1074F000017400017801327901327E0064810064F8
:1075000084FFFF8800028A00019D0A969E00019F69
:10751000FFFFA0013CA2000AA3FFFFA4FFFFA5FFFD
:10752000FFA6FFFFA7FFFFA8FFFFA9FFFF0101784C
:107530001500022F003C4701784802045601044E12
:10754000FFFF58000261FFFF6600028500AF860062
:10755000018700FA890109990006A100FAFAFAFAEE
:1075600001013C1500022F1E3C47017848020456D9
:1075700001034EFFFF58000261FFFF660002850015
:10758000AF8600018700FA890109990000A1000077
:10759000FAFAFA01013C1500002F1E3C47013C4855
:1075A00002035601014EFFFF58000061FFFF660015
:1075B0000085FFFF86FFFF87FFFF8901029900001A
:1075C000A10000FAFAFA0065006F00790083008DCF
:1075D000009700A100AC00B600C000CA00D400DED5
:1075E00000E800F200580060006800700078008039
:1075F00000880090009800A000A800B000B800C16A
:1076000000C800D000D800DF00E600EE00F6004120
:107610000047004D00530059005F0065006C007189
:107620000077007D00830089008F0095009B00A2F9
:1076300000A700AC00B200B900C000C500CA00D26B
:0A76400000D500DD00E100E700EFD7
:103CD80075A71085F97485FA757E017F00E5751260
:103CE800775CE5742FFF50010E8E5A8F5B90001899
:103CF800E0FCA3E0FDEF2DFDEE3CFC8C5C8D5D90BF
:103D08000038E0FAA3E0FBED2BFBEC3AFA8A5C8B77
:103D18005D2275A71085F97485FA757E017F00E527
:103D28007512775CE5742FFF50010E8E5A8F5BACCD
:103D38002DAD2EEF2DFDEE3CFC8C5C8D5D9000389A
:103D4800E0FAA3E0FBED2BFBEC3AFA8A5C8B5D22F0
:103D5800E55DF5FBE55CF5FCD29322E55DF5E9E56B
:103D68005CF5EAD29422E55DF5EBE55CF5ECD291E1
:103D780022E55DF5EDE55CF5EED29222E55DF5FD17
:103D8800E55CF5FED28722E55DF5CEE55CF5CFD2A0
:103D98009022A203B34008E5B54480F5B58006E556
:103DA800B5547FF5B522E50C906FA2F82828730268
:103DB8003E4AA23CB34008E5B54408F5B58006E59F
:103DC800B554F7F5B5807BA23CB34008E5B544028D
:103DD800F5B58006E5B554FDF5B58066A23CB3405F
:103DE80008E5B54410F5B58006E5B554EFF5B5809E
:103DF80051A23CB34008E5B54420F5B58006E5B5C9
:103E080054DFF5B5803CA23CB34008E5B54440F525
:103E1800B58006E5B554BFF5B58027A23CB3400888
:103E2800E5B54480F5B58006E5B5547FF5B5801253
:103E3800A23C9292800CA23C92878006A23C92906F
:023E48008000F8
:106FA200023DB7023DBA023DCF023DE4023DF90285
:106FB2003E0E023E23023E38023E3E023E44023E66
:016FC2004A84
:103E4A00227436900160F07430900161F0742D9004
:103E5A000162F07432900163F07420900164F0748E
:103E6A0036900165F07443900166F07479900167A9
:103E7A00F0746C900168F07420900169F0742090DD
:103E8A00016AF0742090016BF0742090016CF07458
:103E9A002090016DF0742090016EF022900897E056
:103EAA00FEA3E0FF741DD39F74019E400C90741012
:103EBA00120048E493F599804C90F802E493B40513
:103ECA0014900897E0FEA3E0FF907443120048E4C0
:103EDA0093F599803090F802E493D39405401490B6
:103EEA000897E0FEA3E0FF907410120048E493F5EF
:103EFA00998012900897E0FEA3E0FF907476120072
:103F0A0048E493F59990089712776A900897E0FE2B
:103F1A00A3E0FFEFB45007EEB40103754E0022AEE2
:103F2A005AAF5B74068E048F05FF12774C8C5C8D3A
:103F3A005DAE5AAF5B74068E048F05FF1277778CDD
:103F4A005A8D5BC200E55B455A60137406C3955BE4
:103F5A00FFE4955AFE8E5A8F5B785C1277AFE57450
:103F6A00A85CB80015D3955D4010E574C3955DFF54
:103F7A00E4955CFE8E5C8F5D8012E574243CC395EB
:103F8A005DFFE4955CFE8E5C8F5DD200AE5CAF5D3A
:103F9A00743B6F4E6006743C6F4E701AAE5CAF5D38
:103FAA00743B6F4E70057574018003757402755DFC
:103FBA003A755C0080037574002290009DE0B4019C
:103FCA0004C2078002D20790009EE0B40104C2082E
:103FDA008002D2089000DBE075F0D2A4FFAEF07444
:103FEA000A8E048F05FF12774C90088BECF0A3ED34
:103FFA00F09000DBE075F02BA4FFAEF0900014EE19
:10400A00F0A3EFF07E017F00900099E012775C90B8
:10401A0000DCE08E048F05FF12774C740AFF1277DA
:10402A004C8D619000E5E075F0D2A4FFAEF0740A01
:10403A008E048F05FF12774C90088FECF0A3EDF0F9
:10404A009000E7E060139000E7E0F5F0741684FF53
:10405A007E00EF9008EDF0800674649008EDF09011
:10406A0000DDE0900077F0900129E0900084F09064
:10407A00012BE0FE9000D9E08E0088F0A4FFAEF09C
:10408A00EF9008F6F0900104E075F013A4FDACF08F
:10409A00900038ECF0A3EDF0A225B340169001751C
:1040AA00E0700C900176E07006900177E060028083
:1040BA0002C225900175E0B4300F900176E0B44752
:1040CA0008900177E0643B60028004D2268002C235
:1040DA002674E3900076F09000C6E0B40B0874E30F
:1040EA00900076F0805A9000C6E0B419129000DC75
:1040FA00E09075B112008CE493900076F0804190C4
:10410A0000C6E0B41E129000DCE09075CF12008C5D
:10411A00E493900076F080289000C6E0B4281290CC
:10412A0000DCE09075F912008CE493900076F08040
:10413A000F9000C6E0B446089000BDE0900076F00B
:10414A00900096E0FE9008F7E06E601B7599E61203
:10415A00019C74AB900050F012069A7464F50975CC
:10416A0008001205E480FE90008EE070067400904C
:10417A0000C3F090007BE0FE9000C3E0B5066390B8
:10418A00007EE0FE9000E1E0B5065790007CE0FE7C
:10419A009000EFE0B5064B900082E0FE900096E0BA
:1041AA00B5063F90007FE0FE9000D1E0B50633905F
:1041BA00007DE0FE9000DFE0B50627900080E0FE7B
:1041CA009000FCE0B5061B900081E0FE9000FDE047
:1041DA00B5060F900083E0FE90010FE06E700302B7
:1041EA00449490009EE070089000DFE0640460024E
:1041FA00800674039000DFF0900058E0C3940550E5
:10420A00087402900112F0801D9000D1E0D394024C
:10421A0050069000EFE060087406900112F08006E4
:10422A007409900112F0900096E0B40106740090AF
:10423A000096F0900096E0B4020674009000E1F057
:10424A00900096E0B4030674009000EEF09000E14E
:10425A00E0D394014026741B900114F0740090007E
:10426A00AAF074009006DFF074009006E0F0900067
:10427A00C3E0600674009000C3F080329000C3E08F
:10428A00601A7400900114F0741B9000AAF0740074
:10429A009006DFF074009006E0F08012740090013E
:1042AA0014F074009000AAF0741B9006DFF09000DE
:1042BA00D1E0D3940240089000EFE06402600280EB
:1042CA000674009000EFF09000D1E0D39402400809
:1042DA009000EFE0640160028027741C900115F0E1
:1042EA0074009000ABF074009006E3F0740090063E
:1042FA00E4F09000C3E0B4020674019000C3F080B9
:10430A00339000C3E0B4021A7400900115F0741CD3
:10431A009000ABF074009006E3F074009006E4F0AD
:10432A0080127400900115F074009000ABF0741CB8
:10433A009006E3F09000FCE060147407900116F018
:10434A0074009006D7F074009006D8F0800C7400C0
:10435A00900116F074079006D7F09000FDE0601403
:10436A007408900117F074009006DBF07400900650
:10437A00DCF0800C7400900117F074089006DBF0F2
:10438A0090010FE06014742A900787F07400900679
:10439A00D3F074009006D4F0800C7400900787F074
:1043AA00742A9006D3F09000D1E0B402069000EF90
:1043BA00E06002802674049006E7F074059006EB2C
:1043CA00F074069006EFF07400900782F074009083
:1043DA000783F07400900784F0803674009006E733
:1043EA00F074009006E8F074009006EBF074009008
:1043FA0006ECF074009006EFF074009006F0F0748A
:10440A0004900782F07405900783F074069007847D
:10441A00F09000DFE0D394024014741890077AF009
:10442A00741990077BF0741A90077CF0801274005C
:10443A0090077AF0740090077BF0740090077CF084
:10444A00D2249000C3E090007BF09000EFE090004F
:10445A007CF09000E1E090007EF09000D1E09000C6
:10446A007FF09000DFE090007DF0900096E09000F1
:10447A0082F09000FCE0900080F09000FDE0900057
:10448A0081F090010FE0900083F09000F9E0B40110
:10449A0017900024740FF0A374FFF0900026E4F044
:1044AA00A3F074029000F9F09000F9E0B40341908F
:1044BA000026E0FEA3E0FF900024E0FCA3E0FD124A
:1044CA0077A7741012775C7408120039EF9000F81D
:1044DA00F0EF700674FF9000F8F074009000F9F0A5
:1044EA00900025E09000AFF0900024E09000B0F03A
:1044FA0090008AE0900087F0900089E0900086F0B2
:10450A009000B8E0C3941E50569000B8E0F404241A
:10451A001E900088F0900088E075F00684FF7E0007
:10452A008F74900088E075F00684ADF07C008D757C
:10453A00900086E0D39575400D900086E0C395758E
:10454A00900086F0800F900086E02406C39575904F
:10455A000086F00574900087E02574900087F0903B
:10456A000087E0900046F0900046E024149000474F
:10457A00F0900046E02428900048F0900046E0D3EE
:10458A009478400B900046E0C39478900046F090EF
:10459A000047E0D39478400B900047E0C3947890AA
:1045AA000047F0900048E0D39478400B900048E030
:1045BA00C39478900048F0C228900046E0D3943C17
:1045CA00400D900046E0C3943C900046F0D228C2C9
:1045DA0029900047E0D3943C400D900047E0C394F3
:1045EA003C900047F0D229C22A900048E0D3943C7C
:1045FA00400D900048E0C3943C900048F0D22A90C5
:10460A00004CE4F0900046E0643B6007900046E00E
:10461A00B43C20900046E0B43B06740290004CF093
:10462A00900046E0B43C0690004C7401F0900046BD
:10463A007401F090004DE4F0900047E0643B60079D
:10464A00900047E0B43C20900047E0B43B06740277
:10465A0090004DF0900047E0B43C0690004D740184
:10466A00F09000477401F090004EE4F0900048E0AA
:10467A00643B6007900048E0B43C20900048E0B4F6
:10468A003B06740290004EF0900048E0B43C06905D
:10469A00004E7401F09000487401F090008AE0FE28
:1046AA009000EDE02E900051F0900051E0D3943C40
:1046BA00400B900051E0C3943C900051F09000519F
:1046CA00E0D3943C400B900051E0C3943C900051DD
:1046DA00F09000C8E0B40163900051E0641E6007E6
:1046EA00900051E0B43C06900051E004F090005173
:1046FA00E0641D6007900051E0B43B06900051E071
:10470A0014F0900051E0D3943C400B900051E0C368
:10471A00943C900051F0900051E0D3941E400D90CB
:10472A000051E0C3941E900052F0800A900051E0BC
:10473A00241E900052F0755E1E8079900051E0644C
:10474A0014600F900051E064286007900051E0B4B3
:10475A003C06900051E004F0900051E06413600FB1
:10476A00900051E064276007900051E0B43B069046
:10477A000051E014F0900051E0D3943C400B9000BB
:10478A0051E0C3943C900051F0900051E0D394144E
:10479A00400B900051E0C39414900051F0900051E6
:1047AA00E0D39414400B900051E0C394149000514C
:1047BA00F0755E1490008AE0FE9000D0E0D39E501F
:1047CA001390008AE0FE9000D0E0F4042E049000DA
:1047DA0049F0801390008AE02478FE9000D0E0F43B
:1047EA00042E04900049F0900049E075F01484AF5B
:1047FA00F07E00EF4E7006900049E004F090004908
:10480A00E00475F01484AFF07E00EF4E700690005D
:10481A0049E014F0900049E0B47906900049740127
:10482A00F0900049E0D3943C400F900049E0C394D3
:10483A003C900049F0D21F8002C21F900049E02438
:10484A001490004AF0900049E0242890004BF09020
:10485A00004AE0D3943C400B90004AE0C3943C9059
:10486A00004AF090004BE0D3943C400B90004BE0A0
:10487A00C3943C90004BF012019C22C293C294C292
:10488A0091C292C287C290E5B554EFF5B5E5B55429
:10489A00DFF5B5C296C295C2A0C297C2A2C2A1E56F
:1048AA00B554BFF5B5E5B5547FF5B5E5B554FBF597
:1048BA00B5C209755F469000D3E07005756E028037
:1048CA0003756E0375550075540090000C74FFF063
:1048DA00A374DCF0C20FC212C21574C890003AF079
:1048EA0074C890003EF074C8900042F07553007589
:1048FA005200C204754700E570B413037570007561
:10490A00640090001AE4F0A3F0757110C20CC20D95
:10491A00C20EC20375570075560090000EE4F0A34C
:10492A00F0900010E4F0A3F0C22C755900755800FD
:10493A00900095E075F032A4FFAEF0900022EEF000
:10494A00A3EFF0900085E4F09008F3E4F0C227D2D8
:10495A001CC21BD21DC21EC21FC220900012E4F04C
:10496A00A3F022755B00755A00AE5AAF5B741CC384
:10497A009F74019E5003024A61907410120048E429
:10498A0093645F6023907410120048E493647E601D
:10499A0017907410120048E4936481600B907410AD
:1049AA00120048E493B48403024A41AE5AAF5B90C2
:1049BA007410120048E49390008912778D0FBF009B
:1049CA00010EE0FC907410120048ECFEE493FFEE36
:1049DA00C39F5026AE5AAF5B0FBF00010E907410F2
:1049EA00120048AE5AAF5BE493FC90741012004870
:1049FA00E49390008912778DECF0AE5AAF5B907415
:104A0A0010120048E49390008912778DE0FC9074AC
:104A1A0012120048ECFCE493FDECD39D401990740B
:104A2A0012120048E493FC907410120048E4939028
:104A3A00008912778DECF0AE5AAF5B74022FFF50EB
:104A4A00010E8E5A8F5B785B740126F6500418E4C7
:104A5A0036F6400302497322755B00755A00AE5A56
:104A6A00AF5B7432BE00039F5003024B2F90752D2B
:104A7A00120048E49390008912778D0FBF00010E4F
:104A8A00E0FC90752D120048ECFEE493FFEEC39F04
:104A9A005026AE5AAF5B0FBF00010E90752D120063
:104AAA0048AE5AAF5BE493FC90752D120048E4932C
:104ABA0090008912778DECF0AE5AAF5B90752D128B
:104ACA000048E49390008912778DE0FC90752F12CC
:104ADA000048ECFCE493FDECD39D401990752F122D
:104AEA000048E493FC90752D120048E493900089E5
:104AFA0012778DECF0AE5AAF5B742D6F4E7006755F
:104B0A005B33755A00AE5AAF5B74022FFF50010E29
:104B1A008E5A8F5B785B740126F6500418E436F6D9
:104B2A004003024A6822755B00755A00AE5AAF5BB1
:104B3A007432BE00039F5003024BFD907560120051
:104B4A0048E49390008912778D0FBF00010EE0FCB4
:104B5A00907560120048ECFEE493FFEEC39F502666
:104B6A00AE5AAF5B0FBF00010E907560120048AEDF
:104B7A005AAF5BE493FC907560120048E49390008E
:104B8A008912778DECF0AE5AAF5B907560120048CF
:104B9A00E49390008912778DE0FC907562120048C8
:104BAA00ECFCE493FDECD39D401990756212004829
:104BBA00E493FC907560120048E4939000891277A0
:104BCA008DECF0AE5AAF5B742D6F4E7006755B3389
:104BDA00755A00AE5AAF5B74022FFF50010E8E5AFF
:104BEA008F5B785B740126F6500418E436F64003AE
:104BFA00024B3622755B00755A00AE5AAF5B7432AF
:104C0A00BE00039F5003024CCB907593120048E4F8
:104C1A009390008912778D0FBF00010EE0FC90750A
:104C2A0093120048ECFEE493FFEEC39F5026AE5A5F
:104C3A00AF5B0FBF00010E907593120048AE5AAFDA
:104C4A005BE493FC907593120048E49390008912F8
:104C5A00778DECF0AE5AAF5B907593120048E493EF
:104C6A0090008912778DE0FC907595120048ECFC53
:104C7A00E493FDECD39D4019907595120048E49396
:104C8A00FC907593120048E49390008912778DEC9A
:104C9A00F0AE5AAF5B742D6F4E7006755B33755A62
:104CAA0000AE5AAF5B74022FFF50010E8E5A8F5B13
:104CBA00785B740126F6500418E436F64003024C79
:104CCA00042275A71085F97485FA757E017F00E5BF
:104CDA007512775CE5742FFF50010E8E5A8F5BAC0C
:104CEA005CAD5DEF2DFDEE3CFC8C5C8D5D123D589C
:104CFA00123D63123D6E9000D1E0D3940240091236
:104D0A003D79123D84123D8F75A7002285F974857D
:104D1A00FA757E017F00E57512775CE5742FFF5006
:104D2A00010E8E5A8F5B7E017F7690010EE012771C
:104D3A005CAC5AAD5BED2FFFEC3EFE8E5C8F5DE501
:104D4A005DF5EDE55CF5EE900077E4F07412900005
:104D5A0054F02285F97485FA757E017F00E5751293
:104D6A00775CE5742FFF50010E8E5A8F5B9000140A
:104D7A00E0FCA3E0FDEF2DFDEE3CFC8C5C8D5DE5D7
:104D8A005DF5FDE55CF5FE22056522A2DBB3400870
:104D9A009000DDE0900077F0A2DCB34048A2965084
:104DAA00067419900054F0A2955006741990005494
:104DBA00F0A2A050067419900054F0A297500674FD
:104DCA0019900054F0A2A250067419900054F0A24F
:104DDA00A150067419900054F0C296C295C2A0C29E
:104DEA0097C2A2C2A175D8402285A77375A7109051
:104DFA0000D1E0D3940250079000EFE0B40252A22F
:104E0A00D8B34002C293A2D9B34002C294A2DAB381
:104E1A004002C2919000D1E0640260079000D1E0A4
:104E2A00B40417A2DBB34002C292A2DCB34002C2AE
:104E3A0087A2DDB34002C2908015A2D8B34002C255
:104E4A0092A2D9B34002C287A2DAB34002C29080CA
:104E5A002DA2D8B3400AC2939000EFE06002C2923A
:104E6A00A2D9B3400AC2949000EFE06002C287A2BE
:104E7A00DAB3400AC2919000EFE06002C29075D89E
:104E8A00408573A72290F800E4936406600280FECE
:104E9A0012009E75A70075D80075D90475DD0975CD
:104EAA00DE0975D84075A71075D80075D90475DA6A
:104EBA000975DB0975DC0975DD0975DE0975DF0918
:104ECA0075D84075A7001200FB74C8F5097508006B
:104EDA001205E475A70FE5FC900063F0E5FB90006E
:104EEA0064F0E5FA900065F0E5F9900066F075A7C0
:104EFA000090F800E493F5281207039008A0E0D385
:104F0A00940350079008A0E0B4010674009008A02A
:104F1A00F09008A0E09008F7F074019000D2F090A9
:104F2A0008A0E0906FC3F8282873802A802875A704
:104F3A000F75F30F75A700A2A3400674029000D262
:104F4A00F0801375A70F75F31775A700A2A4400682
:064F5A0074029000D2F089
:0C6FC300024F34024F36024F38024F4D8F
:104F60009000D2E0B4022AC21A120AAC7402900075
:104F7000D2F09008A0E0906FCFF8282873801080BE
:0F4F80000E74009000E1F0800674009000EEF0D7
:0C6FCF00024F7D024F7F024F81024F896C
:104F8F008028D21A1209C174019000D2F09008A0A3
:104F9F00E0906FDBF82828738010800E740090006B
:0A4FAF00E1F0800674009000EEF0BF
:0C6FDB00024FA7024FA9024FAB024FB3B8
:104FB90090F807E493900070F0900070E044089036
:104FC9000070F0900070E054FE900070F012039DA4
:104FD900123E4B9008ADE0900175F09008AEE0905C
:104FE9000176F09008AFE0900177F0900175E070DC
:104FF9000C900176E07006900177E060028004C2AF
:10500900258002D2259000C3E00490007BF012496C
:105019006D90F802E493B40505124B30801290F8B4
:1050290002E493D394054005124A628003124BFEB1
:1050390074009000F9F0123FC4E5B54401F5B57468
:1050490006900056F07400900057F07401900058D3
:10505900F090F802E493900059F090F803E49390EB
:10506900005AF090F804E49390005BF07406900005
:105079005CF0900059E0B40506740590005CF0906E
:105089000059E0B40406740490005CF0741E9000AA
:105099005DF0740390005EF0740690005FF0740791
:1050A900900060F090F805E493900061F090F806A4
:1050B900E493900062F0740090006AF0740090002C
:1050C9006BF0740090006CF0740090006DF0740047
:1050D90090006EF0740090006FF074FF900071F012
:1050E900A2B6B39205A2B3B39206A2A4B39222A226
:1050F900A3B39223900072E4F0757000743A90079C
:1051090089F074FD90078AF0900073E4F0756F01DF
:10511900900054E4F09000D3E0B40106741A9000B2
:1051290054F0C221756400C20AD20BC20375720021
:10513900C224120586756000756C0075620075667B
:1051490032756700756800756900756A00756B00CE
:1051590090001AE4F0A3F0756D00D2B2D2A4D2B0D7
:10516900D2B1D2A3D2A7D2A6D2A5D2B77E017F004F
:105179009000B0E012775C9000AFE02FFF50010E75
:10518900900024EEF0A3EFF0EFD394FFEE940F40DC
:1051990007900024E4F0A3F09000F8E0700674FF93
:1051A9009000F8F09000D3E07005756E02800375E9
:1051B9006E037400900118F07400900119F07429BD
:1051C9009006CFF07415900777F07416900778F071
:1051D9007417900779F0740090077DF074009007B8
:1051E9007EF0740190077FF07402900780F07403D9
:1051F900900781F07400900785F07400900786F09D
:10520900D29CE571D3941040037571109006D0E0DB
:10521900D3940C400674009006D0F09006D4E0D3E5
:10522900940C400674009006D4F09006D8E0D3940C
:105239000C400674009006D8F09006DCE0D3940C7C
:10524900400674009006DCF09006E0E0D3940C4030
:105259000674009006E0F09006E4E0D3940C400652
:1052690074009006E4F09006E8E0D3940C400674CC
:10527900009006E8F09006ECE0D3940C4006740028
:105289009006ECF09006F0E0D3940C400674009080
:1052990006F0F0D2EC75CF01A298B34005C298127E
:1052A9000C14E54E6006A299B3B340028005C29979
:1052B9001210A3E54F64016005E54FB4040280D5DF
:1052C900C28E7E107F00E56512775CE58D75F01062
:1052D900A4FDACF0EF2DFDEE3CFCE58B75F01084E0
:1052E900FF7E00ED2FFFEC3EFE8E548F55D28E903F
:1052F90000B6E060099000B6E0C3943D40028056D4
:1053090090001C12776A90001CE0FEA3E0FF900059
:105319001EE0FCA3E0FDEFB5053CEEB50438B2187C
:10532900A204B34013A218B34008E5B54404F5B587
:105339008006E5B554FBF5B590001EE0FEA3E0FF3D
:10534900900020E0FCA3E0FDEF2DFDEE3CFC900079
:105359001EECF0A3EDF09000C3E060099000C3E0FB
:10536900C394034003025416122FCEA2044008909E
:1053790000ADE0F546801BE560C3956150057546B3
:1053890000800F90009AE0C3956250069000C0E03B
:10539900F546E54675F002A4FFAEF0900895EEF0EB
:1053A900A3EFF0AC2FAD30EDD39FEC9E402CE5B5CB
:1053B90054BFF5B59006D0E07006E5B554F7F5B5DC
:1053C9009000C3E0B402099000E1E0C394024002F6
:1053D9008006E5B54480F5B58033900072E0C3944A
:1053E90041502AE5B54440F5B59006D0E07006E590
:1053F900B54408F5B59000C3E0B402099000E1E0B6
:10540900C3940240028006E5B5547FF5B59000C308
:10541900E0B403241230E9AE2FAF30900895E0FCD8
:10542900A3E0FDEFD39DEE9C4008E5B54440F5B5FA
:105439008006E5B554BFF5B590009EE06009A2B3BA
:10544900300601B3B340028056A2B3300601B3401F
:105459004EA2B3300801B34039A21C4030900084F9
:10546900E0D3955F40259008F3E07013900085E044
:10547900B401069008F37401F0900085E004F0A2ED
:105489001BB34005900085E4F0D21BD21CA208B3DF
:105499009206A208B330B301B34004A2089206A24F
:1054A900B6300501B35003025BE0A2B6300501B383
:1054B9005003025BE0A2B6300701B35003025AFE63
:1054C900756F009000B6E0B43D13A207B34008E53C
:1054D900B554FBF5B58006E5B54404F5B5055FA2FD
:1054E90009B3B35013AE54AF5590000CE0FCA3E0E0
:1054F900FDEDC39FEC9E40030256C9E56EB4032E31
:10550900A22CB34022E55FB43B03756E01E55FC38E
:10551900943B50069000547401F0E55FD3943B40EE
:10552900067402900054F0755F01D22C8066E56E16
:10553900B4020A756E01755F3BC21BC21DE55FB4FB
:105549003B05755F01804D900054E07038E55FC3FD
:10555900943B50069000547401F0E55FD3943B40AE
:10556900067402900054F0E55FC3943B5002D221C7
:10557900E55FD3943B4002D221C296C295C2A0C234
:1055890097C2A2C2A19000D3E0B401051248858058
:1055990003755F01AE56AF57AC54AD55EF2DFDEE17
:1055A9003CFC74028C068D071200398E568F579079
:1055B90000B6E060099000B6E0C3943D4002804324
:1055C90090001CE0FEA3E0FF9000B6E08E048F057A
:1055D900FF12774C74018C068D0712003990002058
:1055E900EEF0A3EFF0900020E0F8A3E090001EC8D1
:1055F900F0A3C8F090001CE4F0A3F0C218E5B5547C
:10560900FBF5B5A2A4B34002C222A2A3B34002C2D1
:1056190023A221B34002C221B21E9008F3E0B401D3
:1056290011A21BB34004D21E8002C21E740290084C
:10563900F3F09008F3E0C394025006A204B3B34018
:1056490002800674029008F3F09000DFE0640460C1
:10565900079000D1E0B4046290009EE060069008D3
:10566900F3E07002800DA21D301B01B340059000CC
:1056790085E4F09000D3E064016006A227B3B3503B
:105689001790009EE06009A21B301D01B3B34002D0
:1056990080067405900054F0B21DA21CB3401BA2F1
:1056A9001BB34004D21D8002C21D9000D3E07006D6
:1056B9009008F3E070028002D227C21BC21C803A14
:1056C900AE56AF57AC54AD55EF2DFDEE3CFC740111
:1056D9008C068D071200398E568F57E56EC39402DA
:1056E900500DAC54AD5574B8C39D740B9C400280E9
:1056F900091248857406900054F0E55FB43B1274B2
:1057090003900054F0D2219000D3E0B40103124871
:1057190085AE58AF59AC54AD55EF2DFDEE3CFC8C20
:10572900588D59AE54AF55EFD39DEE9C4011900062
:1057390012E0FAA3E0FBEBC394E8EA940340028089
:105749000690001212776A900010E0FEA3E0FFAC09
:1057590054AD55EF2DFDEE3CFC900010ECF0A3ED9F
:10576900F09000D3E0B40118AE54AF557405127728
:105779005C740112003990000CEEF0A3EFF0801177
:10578900AE54AF55740212775C90000CEEF0A3EFA3
:10579900F0C28E758D00758B0075650075550175A4
:1057A9005400D28EE55F240E75F00F84AFF07E00B1
:1057B900EF4E6003025842E56E6013AE56AF577460
:1057C9000F12775C90000EEEF0A3EFF0800F9000BF
:1057D90010E0F8A3E090000EC8F0A3C8F090000E06
:1057E900E0FEA3E0FFEF4E600B7C797DC212764AA2
:1057F9008E528F53900010E4F0A3F0AE52AF537461
:1058090028BE00039F5010E5642FFF50010E74015C
:105819001200398E528F538553649000DAE0A852F2
:10582900B8000DD395534008E553900053F0800913
:105839009000DAE014900053F09000D1E0B404082D
:10584900900049E0655F6002800EA21E301F01B31F
:105859004004D2208002C220E55F640B6005E55F49
:10586900B429099000C3E06003122C849000C8E0B9
:10587900B40114900051E0655F6007900052E0B5F3
:105889005F03757000801E900051E0655F601390A2
:105899000051E02414655F6009900051E02428B5A7
:1058A9005F03757000A20A5003025A219000DFE0DD
:1058B900C394045006A209B3B3400302596C900083
:1058C9008FE0B40173900111E0B4021412124490F4
:1058D9000078E075F0BCA4FFAEF08E5C8F5D805659
:1058E900E56875F00A84FF7E00900589120048E09A
:1058F900F55B755A00AE5AAF5B9000B4E012775C65
:1059090074648E048F05FF12774C8C5C8D5DE55DA8
:1059190090004FF0AE5AAF5B90008DE012775C7447
:10592900648E048F05FF12774C74BC8C068D0712A8
:10593900775C8E5C8F5D801790008DE075F0BCA45C
:10594900FFAEF08E5C8F5D9000B4E090004FF0E503
:1059590062C394CC5006E55D455C70028003124C2D
:10596900CCD20A9000DFE0B404069008F3E070039B
:10597900025A2190008FE0B40173900111E0B40242
:1059890014121244900078E075F0BCA4FFAEF08EBA
:105999005C8F5D8056E56875F00A84FF7E0090058E
:1059A90089120048E0F55B755A00AE5AAF5B90006A
:1059B900B4E012775C74648E048F05FF12774C8C07
:1059C9005C8D5DE55D90004FF0AE5AAF5B90008D48
:1059D900E012775C74648E048F05FF12774C74BCF7
:1059E9008C068D0712775C8E5C8F5D801790008D19
:1059F900E075F0BCA4FFAEF08E5C8F5D9000B4E062
:105A090090004FF0E562C394CC5006E55D455C70AB
:105A1900028003124CCCD20AE56EB40106E55F643C
:105A290011600280189000DFE0B4040575710380ED
:105A3900097571009000557401F0756E00E56E608E
:105A490003025AF99000D6E0600D900077E0A85261
:105A5900B800069553400280409000D6E0B4021F7A
:105A6900900046E0655F600F900047E0655F600762
:105A7900900048E0B55F03757103756D00800CC235
:105A890001756D0090001AE4F0A3F0900077E060D2
:105A9900067409900054F08057900046E0655F60F5
:105AA9000F900047E0655F6007900048E0B55F40F0
:105AB9009000DFE0B4040FA227B3400575710080A0
:105AC900037571038003757100900046E0B55F06A8
:105AD9009000557401F0900047E0B55F067402909C
:105AE9000055F0900048E0B55F067403900055F04A
:105AF900A207B39205A207B330B601B35003025B04
:105B0900E0756F019000B6E0B43D13A207B34008F9
:105B1900E5B54404F5B58006E5B554FBF5B5E5B53D
:105B29004401F5B5742B900072F0A2079205E55F68
:105B3900D3944A4014D209E55FD39485400B740588
:105B4900900054F0D221755F469000DEE0B4010761
:105B5900E56BC3944140028018E56BC39414500867
:105B69007413900054F08006740E900054F012489B
:105B79008590005CE0FE900059E0C39E40099000CA
:105B890059E0D39408400974FB900054F0124885F9
:105B990090005AE0601590005AE0FE900058E06EBF
:105BA900600974FC900054F012488590005BE06035
:105BB9001590005BE0FE90005DE06E600974FE9058
:105BC9000054F01248859008A0E0600690010EE0AC
:105BD90060028003120B97A221B3400CC296C295B2
:105BE900C2A0C297C2A2C2A190010EE0600CAE523F
:105BF900AF537414BE00059F40028037900096E0B1
:105C0900906FE7F8282873802A8028A2A3B350054B
:105C1900A223B340028005124D16D2238015A2A4F7
:105C2900B35005A222B340028005124D16D222803C
:035C3900028000E6
:106FE700025C10025C12025C14025C27025C3A022B
:026FF7005C3C00
:105C3C00A20CB3B35008900049E0655F6003025DAD
:105C4C00AAA202B35006A201B3B34003025DA49012
:105C5C0000D1E0B404028003025D68123CD89008C5
:105C6C00F3E0B402028003025D56A220B3406790B9
:105C7C000122E0601F900018E0FEA3E0FF90011AE3
:105C8C00E012775C74C88E048F05FF12774C8C5C25
:105C9C008D5D800A900018E0F55CA3E0F55DAE5CCC
:105CAC00AF5D745E12775C74058E048F05FF1277FE
:105CBC004CAE5AAF5BED2FFFEC3EFE8E5C8F5D90D1
:105CCC000038E0FCA3E0FDEF2DFDEE3CFC8C5C8D80
:105CDC005D123D588068900122E0D39403401F90E0
:105CEC000018E0FEA3E0FF90011DE012775C74C881
:105CFC008E048F05FF12774C8C5C8D5D800A9000B2
:105D0C0018E0F55CA3E0F55DAE5CAF5D745E1277F8
:105D1C005C74058E048F05FF12774CAE5AAF5BEDA9
:105D2C002FFFEC3EFE8E5C8F5D900038E0FCA3E014
:105D3C00FDEF2DFDEE3CFC8C5C8D5D123D799000F1
:105D4C00EFE0B40103123D9A8010123D58123D79D8
:105D5C009000EFE0B40103123D9A8039123CD81246
:105D6C003D589000D1E0B4030ED2929000EFE0B415
:105D7C000103123D9A801E9000EFE0B40206123D22
:105D8C001A123D799000EFE0B40106A203B3B340C0
:105D9C00028002D29275A700C20CD20DD20EA20DB7
:105DAC00B3B3500890004AE0655F6003025F2BA21A
:105DBC0002B35006A201B3B34003025F259000D199
:105DCC00E0B404028003025ED9123CD89008F3E0E0
:105DDC00B402028003025EC7A220B3406A90012283
:105DEC00E0D39401401F900018E0FEA3E0FF900167
:105DFC001BE012775C74C88E048F05FF12774C8CF5
:105E0C005C8D5D800A900018E0F55CA3E0F55DAE5A
:105E1C005CAF5D745E12775C74058E048F05FF12A7
:105E2C00774CAE5AAF5BED2FFFEC3EFE8E5C8F5D78
:105E3C00900038E0FCA3E0FDEF2DFDEE3CFC8C5C0B
:105E4C008D5D123D638068900122E0D39404401F65
:105E5C00900018E0FEA3E0FF90011EE012775C7446
:105E6C00C88E048F05FF12774C8C5C8D5D800A9078
:105E7C000018E0F55CA3E0F55DAE5CAF5D745E12FE
:105E8C00775C74058E048F05FF12774CAE5AAF5BAE
:105E9C00ED2FFFEC3EFE8E5C8F5D900038E0FCA396
:105EAC00E0FDEF2DFDEE3CFC8C5C8D5D123D849095
:105EBC0000EFE0B40103123D9A8010123D63123DD5
:105ECC00849000EFE0B40103123D9A8049123CD853
:105EDC00123D639000EFE0C394025007A203B3405D
:105EEC0002D2879000D1E0B4030ED2879000EFE08D
:105EFC00B40103123D9A801E9000EFE0B40206122A
:105F0C003D1A123D849000EFE0B40106A203B3B336
:105F1C0040028002D28775A700D20CC20DD20EA20D
:105F2C000EB3B3500890004BE0655F60030260ACA9
:105F3C00A202B35006A201B3B340030260A69000C4
:105F4C00D1E0B40402800302605A123CD89008F3EA
:105F5C00E0B402028003026048A220B3406A9001C0
:105F6C0022E0D39402401F900018E0FEA3E0FF90C3
:105F7C00011CE012775C74C88E048F05FF12774CFD
:105F8C008C5C8D5D800A900018E0F55CA3E0F55DFB
:105F9C00AE5CAF5D745E12775C74058E048F05FF8A
:105FAC0012774CAE5AAF5BED2FFFEC3EFE8E5C8F42
:105FBC005D900038E0FCA3E0FDEF2DFDEE3CFC8C89
:105FCC005C8D5D123D6E8068900122E0D39405409B
:105FDC001F900018E0FEA3E0FF90011FE012775C19
:105FEC0074C88E048F05FF12774C8C5C8D5D800A13
:105FFC00900018E0F55CA3E0F55DAE5CAF5D745EFF
:10600C0012775C74058E048F05FF12774CAE5AAF75
:10601C005BED2FFFEC3EFE8E5C8F5D900038E0FC5C
:10602C00A3E0FDEF2DFDEE3CFC8C5C8D5D123D8FF5
:10603C009000EFE0B40103123D9A8010123D6E12F5
:10604C003D8F9000EFE0B40103123D9A8049123C61
:10605C00D8123D6E9000EFE0C394025007A203B338
:10606C004002D2909000D1E0B4030ED2909000EF99
:10607C00E0B40103123D9A801E9000EFE0B40206DA
:10608C00123D1A123D8F9000EFE0B40106A203B34B
:10609C00B340028002D29075A700D20CD20DC20E72
:0D60AC00E571906FF9F82828739000F6E078
:036FF9000260B57E
:1060B900907086F82828731225CF80121225CF8078
:0E60C9000D12265980081227058003122705A4
:0F7086000260C00260C50260CA0260CF0260D41F
:1060D7007571010266101228311229487571020282
:1060E7006610122CC8A204B340139000DBE075F0D1
:1060F7001DA4FFAEF0900014EEF0A3EFF090088916
:10610700E0FEA3E0FF740A12775C90000EE0FCA3A8
:10611700E0FD74098F02FF12774C8D078C038E0404
:106127008A058B0612764A90088DEEF0A3EFF09061
:1061370000DFE0B401087450BE00059F4002800DE7
:10614700745090088DF8E4F0E8A3F0801B90088D58
:10615700E0FEA3E0FF74F0BE00039F500B74F090C5
:10616700088DF8E4F0E8A3F0E53770037537019080
:10617700088DE0FEA3E0FFE5372FFF50010E9008E2
:106187008DEEF0A3EFF0757103A233401A9000551E
:01619700E027
:066FFC000260DD0260E905
:10619800907095F8282873800D75710A80087571BC
:0661A8000B800375710C71
:0C70950002619F0261A10261A60261ABD2
:1061AE000266109006D0E060077401F508122DF615
:1061BE00A235B3B35008900787E0642A60028009C5
:1061CE00E5B54402F5B50262789000C4E0D39402BE
:1061DE004045900098E02403A852B800049553500F
:1061EE000990009AE0D395625002800ED202A22B43
:1061FE0040067408900054F0D22B900098E0A852FC
:10620E00B80005D39553500B90009AE02403C39524
:10621E00625002C2028053900098E02403A852B844
:10622E00000495535010E560C39561500990009A93
:10623E00E0D395625002800ED202A22B4006740863
:10624E00900054F0D22B900098E0A852B80005D3DD
:10625E0095535014E561240FC39560400B90009A3E
:10626E00E02403C395625002C202A2024002C22B76
:10627E00A235B3500DA202B35008900787E0642AEE
:10628E0060028006E5B554FDF5B59000DEE07007BE
:10629E00E56BC3941440028002D2029000D3E0B4A6
:1062AE000102D202A2024005757104800A757110B6
:0E62BE0090001AE4F0A3F00266109000C4E015
:067002000261B10262C848
:1062CC009070A1F828287312135A801212135A8056
:0E62DC000D12150D80081215C480031215C492
:0F70A1000262D30262D80262DD0262E20262E79B
:1062EA009006D4E060077402F508122DF675710560
:1062FA0002661012171D7571069006D8E0600774C1
:10630A0003F508122DF69006DCE060077404F50820
:10631A00122DF602661090004FE06006A204B3B395
:10632A004002800DE55FD39414500690004FE014AC
:10633A00F01219A67571079006E0E060077405F57A
:10634A0008122DF69006E4E060077406F508122D8F
:10635A00F6026610900111E0B402031212CB121E6B
:10636A000E7571089006E8E060077407F508122DAB
:10637A00F69006ECE060077408F508122DF602663E
:10638A0010121EF07571090266101222C8A20CB30F
:10639A005005A20DB340028006D20CD20DD20E7562
:1063AA0071109006F0E060077409F508122DF602E4
:1063BA00661090003CE0C39446500AC296C2977495
:1063CA004690003CF090004CE0B4011DE5372406ED
:1063DA00F53790088DE0FEA3E0FF74062FFF500109
:1063EA000E90088DEEF0A3EFF090004CE0B4021D81
:1063FA00E537240CF53790088DE0FEA3E0FF740C16
:10640A002FFF50010E90088DEEF0A3EFF085375B59
:10641A00755A00900046E0F574123F29E55D900038
:10642A003CF0900006E55AF0A3E55BF0E5749000B5
:10643A003DF0C21090088DE0F55AA3E0F55B90009C
:10644A0046E0F574123F29E55D90003AF0900000AD
:10645A00E55AF0A3E55BF0E57490003BF0A20092E8
:10646A001190004CE06002B211C20F75710302660E
:10647A0010900040E0C3944650139000DFE0B4014E
:10648A0002C296C295C2A27446900040F090004D96
:10649A00E0B4011DE5372406F53790088DE0FEA328
:1064AA00E0FF74062FFF50010E90088DEEF0A3EF67
:1064BA00F090004DE0B4021DE537240CF537900842
:1064CA008DE0FEA3E0FF740C2FFF50010E90088DA3
:1064DA00EEF0A3EFF085375B755A00900047E0F5C0
:1064EA0074123F29E55D900040F0900008E55AF0EB
:1064FA00A3E55BF0E574900041F0C21390088DE0CB
:10650A00F55AA3E0F55B900047E0F574123F29E5E0
:10651A005D90003EF0900002E55AF0A3E55BF0E5DD
:10652A007490003FF0A200921490004DE06002B215
:10653A0014C212757103026610900044E0C39446B7
:10654A0050139000DFE0B40102C296C2A0C2A17447
:10655A0046900044F090004EE0B4011DE537240651
:10656A00F53790088DE0FEA3E0FF74062FFF500177
:10657A000E90088DEEF0A3EFF090004EE0B4021DED
:10658A00E537240CF53790088DE0FEA3E0FF740C84
:10659A002FFF50010E90088DEEF0A3EFF085375BC8
:1065AA00755A00900048E0F574123F29E55D9000A5
:1065BA0044F090000AE55AF0A3E55BF0E574900018
:1065CA0045F0C21690088DE0F55AA3E0F55B9000FD
:1065DA0048E0F574123F29E55D900042F09000040E
:1065EA00E55AF0A3E55BF0E574900043F0A200924F
:1065FA001790004EE06002B217C21575710380064B
:06660A0080048002800004
:107008000262FD02632002635E02638B02639402E4
:1070180063BC02647B02654302660A02660C026670
:047028000E026610DE
:1066100090003AE0B55F0280030266EDA20F40727F
:10662000900000E0FEA3E0FFEF4E6021AE56AF57B2
:10663000900000E0FCA3E0FD12000374068E048FBE
:1066400005FF12774C900000ECF0A3EDF090003BBA
:10665000E0601A900000E0FEA3E0FFAC56AD57EFFB
:106660002DFDEE3CFC900000ECF0A3EDF090003B23
:10667000E0D39401401A900000E0FEA3E0FFAC5686
:10668000AD57EF2DFDEE3CFC900000ECF0A3EDF0DB
:10669000D20FAE54AF55900000E0FCA3E0FDEFC375
:1066A0009DEE9C4048124D5D9000DFE090702CF80C
:1066B0002828738030D296802CD2968028D296D209
:1066C000978022A2114010A228301D01B34004D2AD
:1066D000978002D296800EA228301D01B34004D2CA
:0566E000968002D29734
:0F702C000266B30266B50266B90266BD0266C3AC
:1066E500C20F74C890003AF0A20FB3B350079000E0
:1066F5003AE0B55F028048124D5D9000DFE0907092
:106705003BF82828738030D296802CD2968028D2E8
:1067150096D2978022A2114010A228301D01B340C5
:1067250004D2978002D296800EA228301D01B34074
:0767350004D2968002D29706
:0F703B0002670A02670C02671002671402671AE5
:10673C0074C890003AF0C20F90003CE0B55F028044
:10674C00030267E5A2104072900006E0FEA3E0FF92
:10675C00EF4E6021AE56AF57900006E0FCA3E0FD73
:10676C0012000374068E048F05FF12774C900006FE
:10677C00ECF0A3EDF090003DE0601A900006E0FE16
:10678C00A3E0FFAC56AD57EF2DFDEE3CFC900006A0
:10679C00ECF0A3EDF090003DE0D39401401A900092
:1067AC0006E0FEA3E0FFAC56AD57EF2DFDEE3CFC32
:1067BC00900006ECF0A3EDF0D210AE54AF55900063
:1067CC0006E0FCA3E0FDEFC39DEE9C400CC296C21C
:1067DC0097744690003CF0C210A210B3B3500790CF
:1067EC00003CE0B55F02800CC296C29774469000E4
:1067FC003CF0C21090003EE0B55F0280030268DD01
:10680C00A2124072900002E0FEA3E0FFEF4E602166
:10681C00AE56AF57900002E0FCA3E0FD12000374EB
:10682C00068E048F05FF12774C900002ECF0A3ED5E
:10683C00F090003FE0601A900002E0FEA3E0FFAC95
:10684C0056AD57EF2DFDEE3CFC900002ECF0A3EDA5
:10685C00F090003FE0D39401401A900002E0FEA3B8
:10686C00E0FFAC56AD57EF2DFDEE3CFC900002EC7A
:10687C00F0A3EDF0D212AE54AF55900002E0FCA3A1
:10688C00E0FDEFC39DEE9C4048124D5D9000DFE0B3
:10689C0090704AF82828738030D296802CD295803C
:1068AC0028D295D2A28022A2144010A229301D0118
:1068BC00B34004D2A28002D295800EA229301D01D1
:0968CC00B34004D2958002D2A26F
:0F704A000268A30268A50268A90268AD0268B3D4
:1068D500C21274C890003EF0A212B3B350079000E4
:1068E5003EE0B55F028048124D5D9000DFE090709C
:1068F50059F82828738030D296802CD2958028D2DA
:1069050095D2A28022A2144010A229301D01B340C5
:1069150004D2A28002D295800EA229301D01B34077
:0769250004D2958002D2A20A
:0F7059000268FA0268FC02690002690402690A0F
:10692C0074C890003EF0C212900040E0B55F028047
:10693C00030269DEA2134072900008E0FEA3E0FFA0
:10694C00EF4E6021AE56AF57900008E0FCA3E0FD7F
:10695C0012000374068E048F05FF12774C9000080A
:10696C00ECF0A3EDF0900041E0601A900008E0FE1E
:10697C00A3E0FFAC56AD57EF2DFDEE3CFC900008AC
:10698C00ECF0A3EDF0900041E0D39401401A90009C
:10699C0008E0FEA3E0FFAC56AD57EF2DFDEE3CFC3E
:1069AC00900008ECF0A3EDF0D213AE54AF5590006C
:1069BC0008E0FCA3E0FDEFC39DEE9C40159000DFCA
:1069CC00E0B40102C296C295C2A27446900040F097
:1069DC00C213A213B3B35007900040E0B55F02801E
:1069EC00159000DFE0B40102C296C295C2A27446B3
:1069FC00900040F0C213900042E0B55F02800302A9
:106A0C006ADFA2154072900004E0FEA3E0FFEF4E97
:106A1C006021AE56AF57900004E0FCA3E0FD1200DD
:106A2C000374068E048F05FF12774C900004ECF073
:106A3C00A3EDF0900043E0601A900004E0FEA3E0A8
:106A4C00FFAC56AD57EF2DFDEE3CFC900004ECF086
:106A5C00A3EDF0900043E0D39401401A900004E0C1
:106A6C00FEA3E0FFAC56AD57EF2DFDEE3CFC9000C5
:106A7C0004ECF0A3EDF0D215AE54AF55900004E049
:106A8C00FCA3E0FDEFC39DEE9C4048124D5D9000D1
:106A9C00DFE0907068F82828738030D296802CD272
:106AAC00A08028D2A0D2A18022A2174010A22A3006
:106ABC001D01B34004D2A18002D2A0800EA22A30C4
:0B6ACC001D01B34004D2A08002D2A143
:0F706800026AA5026AA7026AAB026AAF026AB5A2
:106AD700C21574C8900042F0A215B3B350079000D6
:106AE70042E0B55F028048124D5D9000DFE0907094
:106AF70077F82828738030D296802CD2A08028D2AD
:106B0700A0D2A18022A2174010A22A301D01B340B3
:106B170004D2A18002D2A0800EA22A301D01B34068
:076B270004D2A08002D2A1FC
:0F707700026AFC026AFE026B02026B06026B0CDD
:106B2E0074C8900042F0C215900044E0B55F028038
:106B3E0003026BE0A216407290000AE0FEA3E0FF93
:106B4E00EF4E6021AE56AF5790000AE0FCA3E0FD79
:106B5E0012000374068E048F05FF12774C90000A04
:106B6E00ECF0A3EDF0900045E0601A90000AE0FE14
:106B7E00A3E0FFAC56AD57EF2DFDEE3CFC90000AA6
:106B8E00ECF0A3EDF0900045E0D39401401A900094
:106B9E000AE0FEA3E0FFAC56AD57EF2DFDEE3CFC38
:106BAE0090000AECF0A3EDF0D216AE54AF55900063
:106BBE000AE0FCA3E0FDEFC39DEE9C40159000DFC4
:106BCE00E0B40102C296C2A0C2A17446900044F085
:106BDE00C216A216B3B35007900044E0B55F028010
:106BEE00159000DFE0B40102C296C2A0C2A17446A5
:106BFE00900044F0C2169000E1E0B402028003025D
:106C0E006D2C900074E0D395675064900074E0F49E
:106C1E00042567FE9000E4E08E00F5F0E884FF7E28
:106C2E00008F74EFC39410500CEF8574F0A4FDAC7C
:106C3E00F08D7480037574FF900074E0D3957440EA
:106C4E000B900074E0C39574F5728003757200901A
:106C5E0000FFE0D3957240069000FFE0F5729001C0
:106C6E0000E0C395725006900100E0F572807190BD
:106C7E000074E0C39567FE9000E4E08E00F5F0E846
:106C8E0084FF7E008F74EFC39410500CEF8574F068
:106C9E00A4FDACF08D7480037574FF85745B755A1A
:106CAE0000900074E0255BFFAE5A50010E8E5A8F95
:106CBE005B74FFBE0009D39F4005855B7280037530
:106CCE0072FF9000FFE0D3957240069000FFE0F552
:106CDE0072900100E0C395725006900100E0F572CB
:106CEE00A204B3B3500D900075E0FE9000ECE0D31B
:106CFE009E5002800E7407900054F0E5B554BFF517
:106D0E00B5801B75A710E5CDC395724008E5B55447
:106D1E00BFF5B58006E5B54440F5B575A700900002
:106D2E00FCE0605E900106E0A852B8000495535056
:106D3E0017900105E0A852B8000ED3955340099064
:106D4E000107E0D395624002801D75A710E5CDC303
:106D5E0094BF4008E5B554EFF5B58006E5B544108F
:106D6E00F5B575A700801B75A710E5CDC3944040FF
:106D7E0008E5B554EFF5B58006E5B54410F5B575E3
:106D8E00A7009000FDE0605E900109E0A852B800F7
:106D9E000495535017900108E0A852B8000ED395F1
:106DAE0053400990010AE0D395624002801D75A7F9
:106DBE0010E5CDC394BF4008E5B554DFF5B58006A8
:106DCE00E5B54420F5B575A700801B75A710E5CD78
:106DDE00C394404008E5B554DFF5B58006E5B544EB
:106DEE0020F5B575A700E570C39413501DE57075B9
:106DFE00F00284AFF07E00EF4E7005123290800AE2
:106E0E00A2EDB34005C2ED123290AE54AF557410E0
:106E1E00C39F74279E400C900073E0C3945A4003A6
:106E2E00026F9FA209B34009124885740690005460
:106E3E00F0A20BB3500EE562D394334007E562C364
:106E4E0094CC40028041900111E0B402141212441D
:106E5E00900078E075F05EA4FFAEF08E5C8F5D80E2
:106E6E000F90008DE075F05EA4FFAEF08E5C8F5D2E
:106E7E00E55D455C6011E5B54401F5B5742B9000F8
:106E8E0072F0124CCCD20B900073E0D394014007F9
:106E9E00E562C3941A40028002C20B9006D0E060F5
:106EAE00077401F508122DF69006D4E060077402FF
:106EBE00F508122DF69006D8E060077403F5081257
:106ECE002DF69006DCE060077404F508122DF6909E
:106EDE0006E0E060077405F508122DF69006E4E072
:106EEE0060077406F508122DF69006E8E060077448
:106EFE0007F508122DF69006ECE060077408F50809
:106F0E00122DF69006F0E060077409F508122DF6C2
:106F1E00900073E0C3945A5010E570B413099000BA
:106F2E0073E004F0757000803FE570B41303757064
:106F3E0000C28E758D00758B0075650075550175D7
:106F4E005400D28E900072E0C394415008900072AB
:106F5E00E004F080067441900072F0900072E0B48C
:106F6E004106E5B554FEF5B5900073E0D3940140AB
:106F7E0007E56BC3944140028006740E900054F0F6
:106F8E009008A0E0600690010EE060028003120BF4
:046F9E009702529E66
:1070B0000000010001400160018001A001C001E069
:1070C00002000300039603B603D603F40400050090
:1070D0000512052405360548055A056C057E059000
:1070E00005A805C005DE0600061406280646066E3D
:1070F00006AE05CF06EE00FF013F015F017F019F55
:1071000001BF01DF01FF02FF039503B503D503F3C0
:1071100003FF04FF05110523053505470559056BD8
:10712000057D058F05A705BF05CE05F106130627CA
:107130000645066D06AD06ED05DD06FF0FAA0FA597
:107140000F9F0F9A0F940F8D0F870F800F780F717D
:107150000F680F600F570F4E0F450F3B0F300F2575
:107160000F1A0F0E0F020EF50EE80EDB0ECC0EBE40
:107170000EAE0E9F0E8E0E7D0E6C0E5A0E470E3406
:107180000E200E0C0DF70DE20DCB0DB50D9D0D85EE
:107190000D6D0D540D3A0D200D050CE90CCE0CB102
:1071A0000C940C760C580C3A0C1B0BFB0BDB0BBB3A
:1071B0000B9A0B790B570B350B130AF10ACE0AAB5E
:1071C0000A870A640A400A1C09F809D409B0098C24
:1071D00009670943091F08FB08D608B2088E086A28
:1071E0000846082307FF07DC07B90796077307510E
:1071F000072F070D06EC06CA06AA06890669064986
:10720000062A060A05EC05CD05B005920575055858
:10721000053C0520050504EA04CF04B5049C04825E
:107220000469045104390422040B03F403DE03C887
:1072300003B2039D038903750361034D033B0328D8
:107240000316030402F202E102D102C002B002A05E
:10725000029102820273026502570249023C022F28
:1072600002220216020901FD01F201E601DB01D052
:1072700001C601BB01B101A7019D0194018B0182EF
:107280000179017001680160015801500148014114
:1072900001390132012B0125011E01180111010BD9
:1072A000010500FF00FA0FA60FA00F990F920F8B98
:1072B0000F840F7C0F740F6B0F620F580F4E0F432C
:1072C0000F380F2C0F1F0F120F050EF70EE80ED8F8
:1072D0000EC80EB70EA50E930E800E6C0E580E4201
:1072E0000E2C0E150DFD0DE40DCB0DB10D950D7988
:1072F0000D5D0D3F0D200D010CE10CC00C9E0C7CB2
:107300000C590C350C100BEA0BC40B9E0B760B4F73
:107310000B260AFD0AD40AAA0A800A550A2A09FF7E
:1073200009D409A8097C0950092508F908CD08A144
:107330000875084A081E07F307C8079D0773074921
:10734000072006F706CE06A6067E06570630060A72
:1073500005E405BF059B057705540532051004EFCC
:1073600004CE04AE048F047104530435041903FDE4
:1073700003E203C703AD0394037B0363034B0334AE
:10738000031E030802F302DE02CA02B602A3029140
:10739000027F026D025C024C023C022C021D020EB6
:1073A000020001F201E401D701CA01BE01B101A648
:1073B000019A018F0185017A01700166015D015317
:1073C000014A01410139013101290121011901124B
:1073D000010B010400FD00F700F000EA00E400DE0C
:1073E00000D900D300CE00C900C400BF00BA00B568
:1073F00000B100AD00A800A400A0009C0099009579
:107400000091008E008A008700840081007E007B4E
:10009E0075B50075840175A70075FFA075EF069004
:1000AE000050E4F075C91075A70F75A1C775A700AC
:1000BE0075D90075CE0C75A70F75F1FE75F2FF752B
:1000CE00F30775F47875A4BA75A5FF75A60775AE16
:1000DE000075AFFF75D48175D5FF75D6FF75D7FF47
:1000EE0075A70075A20175A14775F8092275E60876
:1000FE0075E71075BC0175BE0475BD6C75BE0775D0
:10010E00BDA075BE0875BD0175BC0075BB1875BC6C
:10011E002075BA0875E88075D11375A70F75E105BE
:10012E0075E20075C7401248857597007597807403
:10013E000A12773C7597C0E5975420700280F875C7
:10014E008F0275A700D2AF75980075A90C75A70F11
:10015E0075AB4375ADFB75AC1E75A71075C91875DB
:10016E00CA0075CB0075C80475A700758912758E07
:10017E0004758C00758A00C2A9D28C758D00758BA2
:10018E0000D2ABD28E75B62075D944C2992290009A
:10019E008BE090089FF0900096E09008A0F0900001
:1001AE0097E09008A1F09000B6E09008A2F09000C1
:1001BE00C3E09008A3F09000D1E09008A4F0900066
:1001CE00DFE09008A5F09000E1E09008A6F0900026
:1001DE00EFE09008A7F09000FCE09008A8F09000E7
:1001EE00FDE09008A9F090010FE09008AAF09001B0
:1001FE0027E09008ACF0900175E09008ADF090010A
:10020E0076E09008AEF0900177E09008AFF09001A4
:10021E000EE09008B0F09000F8E09008B1F0900079
:10022E00AFE09008B2F09000B0E09008B3F090000C
:10023E00AAE09008B4F09000ABE09008B5F0900101
:10024E0014E09008B6F0900115E09008B7F0900118
:10025E0016E09008B8F0900117E09008B9F0900100
:10026E0018E09008BAF09006CFE09008BBF0900628
:10027E00D3E09008BCF09006D7E09008BDF0900651
:10028E00DBE09008BEF09006DFE09008BFF090062D
:10029E00E3E09008C0F09006E7E09008C1F0900609
:1002AE00EBE09008C2F09006EFE09008C3F09006E5
:1002BE00F3E09008C4F0900777E09008C5F090073F
:1002CE0078E09008C6F0900779E09008C7F09007A4
:1002DE007AE09008C8F090077BE09008C9F090078C
:1002EE007CE09008CAF090077DE09008CBF0900774
:1002FE007EE09008CCF090077FE09008CDF090075C
:10030E0080E09008CEF0900781E09008CFF0900743
:10031E0082E09008D0F0900783E09008D1F090072B
:10032E0084E09008D2F0900785E09008D3F0900713
:10033E0086E09008D4F0900787E09008D5F0900101
:10034E0019E09008D6F090011AE09008D7F09001CD
:10035E001BE09008D8F090011CE09008D9F09001B5
:10036E001DE09008DAF090011EE09008DBF090019D
:10037E001FE09008DCF0900120E09008DDF0900185
:10038E0021E09008DEF0900122E09008DFF022904C
:10039E00089FE090008BF09008A0E0900096F090FF
:1003AE0008A1E0900097F09008A2E09000B6F090BF
:1003BE0008A3E09000C3F09008A4E09000D1F09064
:1003CE0008A5E09000DFF09008A6E09000E1F09024
:1003DE0008A7E09000EFF09008A8E09000FCF090E5
:1003EE0008A9E09000FDF09008AAE090010FF090AF
:1003FE0008ACE0900127F09008B0E090010EF0906C
:10040E0008B1E09000F8F09008B2E09000AFF090E4
:10041E0008B3E09000B0F09008B4E09000AAF0901D
:10042E0008B5E09000ABF09008B6E0900114F090A3
:10043E0008B7E0900115F09008B8E0900116F09022
:10044E0008B9E0900117F09008BAE0900118F0900A
:10045E0008BBE09006CFF09008BCE09006D3F09079
:10046E0008BDE09006D7F09008BEE09006DBF09055
:10047E0008BFE09006DFF09008C0E09006E3F09031
:10048E0008C1E09006E7F09008C2E09006EBF0900D
:10049E0008C3E09006EFF09008C4E09006F3F090E9
:1004AE0008C5E0900777F09008C6E0900778F090C6
:1004BE0008C7E0900779F09008C8E090077AF090AE
:1004CE0008C9E090077BF09008CAE090077CF09096
:1004DE0008CBE090077DF09008CCE090077EF0907E
:1004EE0008CDE090077FF09008CEE0900780F09066
:1004FE0008CFE0900781F09008D0E0900782F0904E
:10050E0008D1E0900783F09008D2E0900784F09035
:10051E0008D3E0900785F09008D4E0900786F0901D
:10052E0008D5E0900787F09008D6E0900119F0907A
:10053E0008D7E090011AF09008D8E090011BF090D7
:10054E0008D9E090011CF09008DAE090011DF090BF
:10055E0008DBE090011EF09008DCE090011FF090A7
:10056E0008DDE0900120F09008DEE0900121F0908F
:10057E0008DFE0900122F022754800900897E4F021
:10058E00A3F0753200753100754E00754F00C22F05
:10059E00D2309008A0E06002D22474FE900899F840
:1005AE00E4F0E8A3F074FE90089DF8E4F0E8A3F000
:1005BE0074FE90089BF8E4F0E8A3F0745A9008F1EA
:1005CE00F0745A9008F2F0D231C22DC233C232C248
:1005DE002EC235C23B22750B00750A00AE0AAF0B58
:1005EE00AC08AD09EDC39FEC9E401674FF12773C2C
:1005FE0075CF01780B740126F6500418E436F650C8
:10060E00DB22C2AF75D904758F0375B7A575B7F127
:10061E0090F800E4F0758F0175B7A575B7F1E52870
:10062E0090F800F075B7A575B7F190F801E4F07584
:10063E00B7A575B7F19008E5E090F802F075B7A58B
:10064E0075B7F19008E9E090F803F075B7A575B7A6
:10065E00F19008E6E090F804F075B7A575B7F19043
:10066E0008E7E090F805F075B7A575B7F19008E8C2
:10067E00E090F806F075B7A575B7F19008EAE0902E
:10068E00F807F0758F0075D944D2AF22900050E074
:10069E00B4AB61C2AF75D90475B62275F522758FEC
:1006AE000375B7A575B7F1740090F600F0758F015C
:1006BE00755B00755A00AE5AAF5B7445BE00279F3E
:1006CE00402475B7A575B7F190089F120048E0FC5D
:1006DE0090F600120048ECF0785B740126F6500498
:1006EE0018E436F650D0758F0075F51175B6207575
:1006FE00D944D2AF22C2AF75F52275D904755B000D
:10070E00755A00AE5AAF5B7445BE00229F401F90D3
:10071E00F600120048E493FC90089F120048ECF09B
:10072E00785B740126F6500418E436F650D575D968
:10073E004475F511D2AF22900050E0B4AA028003A6
:10074E00020882C2AF75D90475B62275F522758F6F
:10075E000375B7A575B7F1740090F400F075B7A5E1
:10076E0075B7F1740090F200F075B7A575B7F17416
:10077E000090F000F075B7A575B7F1740090EE001B
:10078E00F0758F01755B00755A00AE5AAF5B74FF42
:10079E00C39F74019E402475B7A575B7F19000896B
:1007AE00120048E0FC90F400120048ECF0785B7404
:1007BE000126F6500418E436F650CF755B00755AD4
:1007CE0000AE5AAF5B74FFC39F74019E402475B791
:1007DE00A575B7F1900289120048E0FC90F2001264
:1007EE000048ECF0785B740126F6500418E436F6F7
:1007FE0050CF755B00755A00AE5AAF5B74FFC39F46
:10080E0074019E402475B7A575B7F1900489120046
:10081E0048E0FC90F000120048ECF0785B74012682
:10082E00F6500418E436F650CF755B00755A00AEDC
:10083E005AAF5B74FFC39F74019E402475B7A575B4
:10084E00B7F1900689120048E0FC90EE00120048C5
:10085E00ECF0785B740126F6500418E436F650CFAF
:10086E00758F0075F51175B62075D944D2AF743AEF
:10087E00900789F022900050E0B4AA02800302098A
:10088E00C0C2AF75D90475B62275F522758F037582
:10089E00B7A575B7F1740090EC00F075B7A575B7F4
:1008AE00F1740090EA00F075B7A575B7F174009079
:1008BE00E800F075B7A575B7F1740090E600F07515
:1008CE008F01755B00755A00AE5AAF5B74FFC39F04
:1008DE0074019E402475B7A575B7F190008912007A
:1008EE0048E0FC90EC00120048ECF0785B740126B6
:1008FE00F6500418E436F650CF755B00755A00AE0C
:10090E005AAF5B74FFC39F74019E402475B7A575E3
:10091E00B7F1900289120048E0FC90EA00120048FC
:10092E00ECF0785B740126F6500418E436F650CFDE
:10093E00755B00755A00AE5AAF5B74FFC39F7401AE
:10094E009E402475B7A575B7F1900489120048E052
:10095E00FC90E800120048ECF0785B740126F6502B
:10096E000418E436F650CF755B00755A00AE5AAFD8
:10097E005B74FFC39F74019E402475B7A575B7F1D4
:10098E00900689120048E0FC90E600120048ECF058
:10099E00785B740126F6500418E436F650CF758F46
:1009AE000075F51175B62075D944D2AF743A90071B
:1009BE0089F022C2AF75D90475F522755B00755AA0
:1009CE0000AE5AAF5B74FFC39F74019E401F90F43C
:1009DE0000120048E493FC900089120048ECF07875
:1009EE005B740126F6500418E436F650D4755B009D
:1009FE00755A00AE5AAF5B74FFC39F74019E401FC1
:100A0E0090F200120048E493FC900289120048EC28
:100A1E00F0785B740126F6500418E436F650D4755F
:100A2E005B00755A00AE5AAF5B74FFC39F74019E94
:100A3E00401F90F000120048E493FC9004891200CD
:100A4E0048ECF0785B740126F6500418E436F65044
:100A5E00D4755B00755A00AE5AAF5B74FFC39F74BA
:100A6E00019E401F90EE00120048E493FC90068910
:100A7E00120048ECF0785B740126F6500418E43648
:100A8E00F650D475F51175D944D2AF74019000D2D9
:100A9E00F0743A900789F09008F87401F022C2AF12
:100AAE0075D90475F522755B00755A00AE5AAF5BA9
:100ABE0074FFC39F74019E401F90EC00120048E427
:100ACE0093FC900089120048ECF0785B740126F6D6
:100ADE00500418E436F650D4755B00755A00AE5AC1
:100AEE00AF5B74FFC39F74019E401F90EA0012001B
:100AFE0048E493FC900289120048ECF0785B740194
:100B0E0026F6500418E436F650D4755B00755A007C
:100B1E00AE5AAF5B74FFC39F74019E401F90E800F6
:100B2E00120048E493FC900489120048ECF0785BC4
:100B3E00740126F6500418E436F650D4755B007531
:100B4E005A00AE5AAF5B74FFC39F74019E401F9054
:100B5E00E600120048E493FC900689120048ECF07F
:100B6E00785B740126F6500418E436F650D475F509
:100B7E001175D944D2AF74029000D2F0743A900736
:100B8E0089F074029008F8F02274019000D2F0906F
:100B9E0008A0E0903C1EF828287380188016A2A3A7
:100BAE00400674029000D2F0800AA2A4400674029D
:040BBE009000D2F0E1
:0C3C1E00020BA8020BAA020BAC020BB8B0
:100BC2009000D2E0B40105A239B34002801AD239B2
:100BD2001248851209C174019000D2F012039D12CD
:100BE2003E4B741B900054F09000D2E0B40206A277
:100BF20039B3B34002801AC239124885120AAC7462
:100C0200029000D2F012039D123E4B741B900054CE
:100C1200F022E54F64046006E59964FF60028031CA
:100C2200A22F4004D22F8027E54F600874E6254F9B
:100C3200900054F0E54E600874F0254E900054F098
:100C4200E54FB4010280FE754F00754E00C22F8041
:100C520002C22FE54F903C2AF8282873754F00E511
:100C620099B4FF03754E01E599B4FE03754E02E592
:100C720099B4FD03754E03E599B4FC03754E04E582
:100C820099B4FA03754E05E599B4FB06754F011246
:100C92004885E599B4F906754F04124885E599B47B
:100CA200F733124885C29C74AB900050F012069A3A
:100CB20074AA900050F09008F8E0B40105120745BC
:100CC2008003120883900050E4F0D29C754F0075A7
:100CD2004E007599F7E599D394E54007E599C394D9
:100CE200F040028016859950754F027E017F00E523
:100CF20050C394E612775C8E338F34900897E4F0F9
:100D0200A3F0E599D394C24007E599C394E6400263
:100D12008028859950754F0374E5C39550F5347555
:100D22003300AE33AF349070B012772BE493F87483
:100D32000193900897C8F0A3C8F0D2990210A2902C
:100D420008ACE0700AA225B35005A226B340028087
:100D52005C900897E0FEA3E0FF74FFBE00039F5083
:100D620009EFC39446EE9406402B900897E0FEA349
:100D7200E0FFEFD3946DEE94064009EFC394EEEEDC
:100D820094064011900897E0FEA3E0FFEFD394FF92
:100D9200EE94064013900897E0FEA3E0FF900089CE
:100DA200120048E599F080038599758011900897A3
:100DB200E0FEA3E0FF900089120048E599F0900858
:100DC2009712776A900897E0FEA3E0FFEFB401065E
:100DD200EEB407028003020E9B900789E0B43C0246
:100DE2008003020E9BA225B35005A226B3400280C7
:100DF20055C29C12039D900096E09008F7F0123FB6
:100E0200C4900175E09008ADF0900176E09008AED4
:100E1200F0900177E09008AFF074AB900050F012C0
:100E2200069A74AA900050F09008F8E0B4010512F6
:100E3200074580031208839008F8E09000D2F090F2
:100E42000050E4F08048C29C12019C74009008ADEE
:100E5200F074009008AEF074009008AFF090009625
:100E6200E09008F7F0123FC474AB900050F0120605
:100E72009A74AA900050F0120745120883D29C750A
:100E820099FB7464F5097508001205E480FED29C92
:100E9200754F00754E007599FB0210A2900897E0FD
:100EA200FEA3E0FFEF4E700685993275310090087F
:100EB20097E0FEA3E0FF74016F4E701BAC31AD32C0
:100EC200AA33AB34ED2BFBEC3AFA8A068B0790007F
:100ED20089120048E599F090089712776A9008976E
:100EE200E0FEA3E0FF74026F4E7021AC31AD3274AC
:100EF200566D4C7006E55064E66002800312488528
:100F0200123FC4855099754F00754E000210A29091
:100F12000897E0FEA3E0FF900089120048E599F0EF
:100F220090089712776A900897E0FEA3E0FFAC332F
:100F3200AD348F028E038C068D079070F612772BDC
:100F4200E493F9740193FEEAD39EEB99400985502C
:100F520099754F00754E000210A2900897E0FEA30B
:100F6200E0FF900089120048E599F0900897127707
:100F72006A900897E0FEA3E0FFEFB40006EEB4012A
:100F82000280030210A2900066E0D394C7400B9047
:100F92000066E0C394C8F551801A900066E0D394CD
:100FA20063400B900066E0C39464F55180069000A4
:100FB20066E0F551E55175F002A4FFAEF08F74EFD3
:100FC20090008912778DEFFCE0FDEC90008C127797
:100FD2008DEDFCE0FDEC2DB5510280030210930F64
:100FE200EF90008912778DE574FFE0FCEF90008DA1
:100FF20012778DECFFE0FCEFC39CB5510280030237
:101002001093E57490008B12778DE574FFE0FCEF8E
:1010120090008E12778DECFFE0FCEF2CB55172E55B
:101022007490008F12778DE0C395519008E5F0E53A
:101032007490009012778DE0C395519008E6F0E528
:101042007490009312778DE0C395519008E7F0E514
:101052007490009412778DE0C395519008E8F0E502
:101062007490009512778DE0C395519008E9F0E5F0
:101072007490009612778DE0C395519008EAF012B1
:1010820006107599F97464F5097508001205E48073
:10109200FE7599FF7464F5097508001205E480FE77
:0F3C2A00020C5E020D41020E9E020F11020F5C92
:1010A20022E54E903C39F828287302118790089760
:1010B200E0FEA3E0FF900056120048E0F599900888
:1010C2009712776A900897E0FEA3E0FF741C6F4EB8
:1010D2007003754E00021187856F9902118790087F
:1010E20097E0FEA3E0FF900089120048E0F599EF37
:1010F200B40107EEB40703754E0090089712776AA1
:07110200021187900898E03C
:0F3C39000210AC0210AF0210DA0210E002110507
:10110900903CABF82828738553998067856099804E
:1011190062856299805D8566998058856899805352
:10112900856999804E856A998049856B9980449033
:10113900001BE0F599803CA230B340077599FAC2CB
:10114900308017A224B3400575990F800B90005485
:10115900E0F599900054E4F0C2248017856C9980D9
:1011690012856799800D856D9980087599FC8003B2
:03117900754E00B0
:103CAB0002111002111502111A02111F0211240226
:103CBB00112902112E021133021138021140021187
:0D3CCB006502116A02116F02117402117975
:0B117C0090089712776A8003123EA6CD
:033C4800021184E2
:1011870022E538255BFFAE5A50010E900089120008
:1011970048E0F539E538255BFFAE5A50010E0FBF21
:1011A70000010E900089120048E0F53A85403CE5C1
:1011B70039B53A058539388041E53AD39539401D27
:1011C700E53AC39539853BF0A4FFAEF0E53C8E04C4
:1011D7008F05FF12774CED2539F538801DE539C3AA
:1011E700953A853BF0A4FFAEF0E53C8E048F05FFF2
:1011F70012774CEDF4042539F53822E53AD39539C1
:10120700401DE53AC39539853BF0A4FFAEF0E53CB8
:101217008E048F05FF12774CED2539F538801DE5D3
:1012270039C3953A853BF0A4FFAEF0E53C8E048FB9
:1012370005FF12774CEDF4042539F5382290008F1D
:10124700E0B4017FE56875F00A84FF7E008F38E51A
:101257006875F00A84ADF07C008D3B75400A755ABD
:1012670005755B24E538C394115005121188800673
:101277009005BEE0F538E538C394F05008E538909E
:101287000078F0800674EF900078F0E56875F00A52
:1012970084FF7E008F38E56875F00A84ADF07C0026
:1012A7008D3B75400A755A05755B5AE538C394112D
:1012B700500512118880069005F4E0F538E538905E
:1012C700004FF02290008FE0B4010280030213590F
:1012D700E56875F00A84FF7E008F38E56875F00AC7
:1012E70084ADF07C008D3B75400A755A05755B36F9
:1012F700E538C39411500512118880069005D0E097
:10130700F538E538C394F0500585384C8003754CA3
:10131700EFE56875F00A84FF7E008F38E56875F0A1
:101327000A84ADF07C008D3B75400A755A05755BE4
:1013370048E538C39411500512118880069005E2DC
:10134700E0F538E538C394F0500585384D800375CE
:101357004DEF22E56075F00484FF7E008F38E5606D
:1013670075F00484ADF07C008D3B754004755A011F
:10137700755B00E538C3943F5005121188800690CD
:1013870001C8E0F538E538900891F8E4F0E8A3F0F3
:10139700900053E075F020A4FFAEF09000DAE08EE5
:1013A700048F05FF12774C8D389000C2E0D395600B
:1013B70050030214659000E6E0D395604010ED906D
:1013C70001C912778DE0F52C752B0002146290008D
:1013D700B1E0D395604043E5389001C912778DE0BD
:1013E700F539E5389001E912778DE0F53A9000E696
:1013F700E0F4042560F53B9000B1E0FE9000E6E0E4
:10140700F4042EF53CE539B53A05853938800312E1
:10141700120285382C752B008041E5389001E912BE
:10142700778DE0F539E53890020912778DE0F53AC6
:101437009000B1E0F4042560F53B9000C2E0FE9017
:1014470000B1E0F4042EF53CE539B53A05853938A5
:10145700800312120285382C752B0002150C9000A0
:10146700E9E0D395605011E53890024912778DE095
:10147700F52C752B0002150C9000B2E0D395605047
:1014870043E53890022912778DE0F539E538900267
:101497004912778DE0F53A9000B2E0F4042560F543
:1014A7003B9000E9E0FE9000B2E0F4042EF53CE545
:1014B70039B53A05853938800312120285382C75FB
:1014C7002B008041E53890020912778DE0F539E568
:1014D7003890022912778DE0F53A9000C2E0F404C3
:1014E7002560F53B9000B2E0FE9000C2E0F4042EC8
:1014F700F53CE539B53A058539388003121202857E
:10150700382C752B00229000FAE0F53D75401175D7
:101517005A02755B00AE52AF53E53D75F00FA4FD5F
:10152700ACF0EDD39FEC9E4021E53D8E048F05FF87
:1015370012774CED75F010A4FFAEF0E56075F01171
:1015470084FD7C00ED2FF53E800EE56075F011847B
:10155700FF7E00EF24F0F53E853E38E56075F0111B
:1015670084AFF07E008F3B12118885383FAE52AFB3
:10157700539000FAE075F00FA4FDACF0EDD39FECAB
:101587009E4028755A02755B10853E381211888572
:101597003F3985383AAE52AF53E53D8E048F05FF8C
:1015A7001277778D3B853D3C121202E53890089102
:1015B700F8E4F0E8A3F0752C64752B00229000FA8C
:1015C700E0F53D754011755A02755B00AE52AF5399
:1015D700E53D75F00FA4FDACF0EDD39FEC9E4021E7
:1015E700E53D8E048F05FF12774CED75F010A4FFD3
:1015F700AEF0E56275F01184FD7C00ED2FF53E80BD
:101607000EE56275F01184FF7E00EF24F0F53E854C
:101617003E38E56275F01184AFF07E008F3B121102
:101627008885383FAE52AF539000FAE075F00FA4AB
:10163700FDACF0EDD39FEC9E4028755A02755B1008
:10164700853E38121188853F3985383AAE52AF53F7
:10165700E53D8E048F05FF1277778D3B853D3C1264
:101667001202E538900891F8E4F0E8A3F0E56C6021
:1016770017E56CC394FE50109000EEE0B402099099
:1016870000DCE0D3940B5002801F900891E0FEA38A
:10169700E0FFE56C12775C74E78E048F05FF127725
:1016A7004C900891ECF0A3EDF09000C4E0B4045F17
:1016B700E56075F00484FF7E008F38E56075F004FF
:1016C70084ADF07C008D3B754004755A01755B0055
:1016D700E538C3943F500512118880069001C8E091
:1016E700F538900891E0FEA3E0FFE53812775C74C7
:1016F700328E048F05FF12774C900891E0FEA3E02D
:10170700FFEF2DFDEE3CFC900891ECF0A3EDF0759A
:101717002C64752B002290008FE0B40146E56875B4
:10172700F00A84FF7E008F38E56875F00A84ADF013
:101737007C008D3B75400A755A05755B00E538C31B
:1017470094115005121188800690059AE0F538AE7D
:101757002BAF2CE5382FFF50010E746412779F8E44
:101767002B8F2C900090E0B40146E56975F00A8450
:10177700FF7E008F38E56975F00A84ADF07C008D37
:101787003B75400A755A05755B6CE538C394115073
:10179700051211888006900606E0F538AE2BAF2CAF
:1017A700E5382FFF50010E746412779F8E2B8F2C14
:1017B70090009FE0B40249E56BC3944175F005843E
:1017C700FF7E008F38E56B75F00584ADF07C008DEA
:1017D7003B754005755A06755B00E538C394135091
:1017E70005121188800690069CE0F538AE2BAF2CC9
:1017F700E5382FFF50010E746412779F8E2B8F2CC4
:101807009000E1E0B4020280030218BCE56075F0C5
:101817001584FF7E008F38E56075F01584ADF07C88
:10182700008D3B754015755A03755BF4E538C39415
:101837000B50051211888006900488E0F538E538CA
:1018470075F0FFA4FFAEF09000E2E08E048F05FF75
:1018570012774CED900074F0E56775F078A4FFAE51
:10186700F074FF8E048F05FF12774C8C5A8D5B74D2
:10187700028C068D071200398F38AC5AAD5B7404A1
:10188700FF1277778D3B754004755A06755B28E51F
:1018970038C3941D500512118880069006CEE0F5D6
:1018A70038AE2BAF2CE5382FFF50010E746412773A
:1018B7009F8E2B8F2C90008EE0B4025DE56275F051
:1018C70064A4FFAEF074081200398E5C8F5D740556
:1018D7008E048F05FF12774C8D38AE5CAF5D7405B3
:1018E7008E048F05FF1277778D3B754005755A0576
:1018F700755BDEE538C39413500512118880069096
:10190700067AE0F538AE2BAF2CE5382FFF50010EE5
:10191700746412779F8E2B8F2C9000D0E0707F908D
:101927000053E075F00A84FF7E008F38900053E083
:1019370075F00A84ADF07C008D3B75400A755A0539
:10194700755BC0E538C3940E500512118880069068
:101957000657E0F538E538900079F09000EFE0B4ED
:10196700023C900053E075F00A84FF7E008F3890A8
:101977000053E075F00A84ADF07C008D3B75400A9A
:10198700755A05755BCFE538C3940E50051211885B
:101997008006900666E0F538E53890007AF02290E8
:1019A7000097E0B401179008ECE0252CFFAE2B5010
:1019B700010E9000EBE012779F8E2B8F2C90010F7A
:1019C700E0B40114900110E0A852B80004955350F8
:1019D70007E560C39561400280139000B9E0252CAC
:1019E700FFAE2B50010E8E2B8F2C021E0D900097F1
:1019F700E0B40306A22DB3B3400280509008F6E08E
:101A070070109008EFE0C39405A852B800069553EC
:101A1700400280109000B9E0252CFFAE2B50010E3C
:101A27008E2B8F2C9008F6E0600D9008EFE0A852FF
:101A3700B800069553400280109000B9E0252CFFAE
:101A4700AE2B50010E8E2B8F2C021E0D900091E0B5
:101A5700B402028003021E0D900094E0602FE56837
:101A6700D394464028900012E0FEA3E0FF9000CFF9
:101A7700E075F003A4FDACF0EFD39DEE9C400E9013
:101A870000F3E0A852B80005D395535003021E0D8A
:101A97009000C4E0B403028003021C5585625B75A5
:101AA7005A0090009BE0A852B800049553500E903E
:101AB700009CE0A85AB80005D3955B5003021C525E
:101AC700E56275F002A4FFAEF074158E048F05FF72
:101AD70012774C8C068D07900619120048FEE0FF1E
:101AE700EE900093E0FEEF8E0088F0A4FFAEF07456
:101AF700648E048F05FF12774C8C5A8D5B900053D0
:101B0700E075F018A4FFAEF09000DAE08E048F05C0
:101B1700FF12774C8C068D07900631120048AE5A9B
:101B2700AF5BE012775C74648E048F05FF12774C0D
:101B37008C5A8D5BE566A85AB80005D3955B5003B0
:101B4700021BC9E566C3955BFFE4955AFE8E5A8F63
:101B57005B7428BE00039F500C755B28755A007490
:101B67000D900054F0AE5AAF5B900094E012775C92
:101B770074288E048F05FF12774C8C5A8D5B900862
:101B870091E0FEA3E0FF740A8E048F05FF12774CE5
:101B97008D068C07AC5AAD5BCFCECF120003740A0B
:101BA7008E048F05FF12774C8C5A8D5B900891E05D
:101BB700FEA3E0FF1277A7900891EEF0A3EFF002E3
:101BC7001C52E566A85AB80004955B507EAE5AAF22
:101BD7005BE56612779F8E5A8F5B7428BE00039F62
:101BE700500C755B28755A00740D900054F0AE5A6E
:101BF700AF5B900094E012775C74288E048F05FF2A
:101C070012774C8C5A8D5B900891E0FEA3E0FF742D
:101C17000A8E048F05FF12774C8D068C07AC5AADE0
:101C27005BCFCECF120003740A8E048F05FF1277A5
:101C37004C8C5A8D5B900891E0FEA3E0FFEF2DFDE1
:101C4700EE3CFC900891ECF0A3EDF0021E0D900025
:101C5700DCE08560F0A4FFAEF0740512775C7407D2
:101C67001200398E5A8F5B90009BE0A852B800048F
:101C77009553501290009CE075F002A4FDACF0EF74
:101C8700C39DEE9C4003021E0DE56075F00B84FFBB
:101C97007E00900619120048FEE0FFEE900093E0E8
:101CA700FEEF8E0088F0A4FFAEF074648E048F05FB
:101CB700FF12774C8C5A8D5B900053E075F018A497
:101CC700FFAEF09000DAE08E048F05FF12774C8CA0
:101CD700068D07900631120048AE5AAF5BE01277C7
:101CE7005C74648E048F05FF12774C8C5A8D5BE50C
:101CF70066A85AB80005D3955B5003021D84E566B4
:101D0700C3955BFFE4955AFE8E5A8F5B7428BE001D
:101D1700039F500C755B28755A00740D900054F0A2
:101D2700AE5AAF5B900094E012775C74288E048FF4
:101D370005FF12774C8C5A8D5B900891E0FEA3E06B
:101D4700FF740A8E048F05FF12774C8D068C07AC43
:101D57005AAD5BCFCECF120003740A8E048F05FFF6
:101D670012774C8C5A8D5B900891E0FEA3E0FF122E
:101D770077A7900891EEF0A3EFF0021E0DE566A895
:101D87005AB80004955B507EAE5AAF5BE566127792
:101D97009F8E5A8F5B7428BE00039F500C755B287B
:101DA700755A00740D900054F0AE5AAF5B900094D2
:101DB700E012775C74288E048F05FF12774C8C5ADB
:101DC7008D5B900891E0FEA3E0FF740A8E048F05F7
:101DD700FF12774C8D068C07AC5AAD5BCFCECF1276
:101DE7000003740A8E048F05FF12774C8C5A8D5BA3
:101DF700900891E0FEA3E0FFEF2DFDEE3CFC90087C
:101E070091ECF0A3EDF0229000EFE0B4027BE560E7
:101E170075F00884FF7E008F38E56075F00884ADA3
:101E2700F07C008D3B754008755A01755BE0E5381D
:101E3700C3943F50051211888006900288E0F53858
:101E4700E538900893F8E4F0E8A3F0900893E0FEF3
:101E5700A3E0FFAC2BAD2C12000374648E048F0536
:101E6700FF12774C900893ECF0A3EDF090008CE014
:101E77008C068D0712775C74648E048F05FF1277CA
:101E87004C900893ECF0A3EDF0900891E0FEA3E0EE
:101E9700FFAC2BAD2C12000374648E048F05FF1268
:101EA700774C900891ECF0A3EDF090008CE08C0655
:101EB7008D0712775C74648E048F05FF12774C9040
:101EC7000891ECF0A3EDF0A204401DAE52AF53749D
:101ED70005BE00039F5002D204E562D394CC4008AC
:101EE700D2027411900054F0229000EEE0B4020880
:101EF7009000DCE0640B60028045900891E0FEA34F
:101F0700E0FFE56C12775C74E78E048F05FF1277AC
:101F17004C900891ECF0A3EDF09000EFE0B4021FB5
:101F2700900893E0FEA3E0FFE56C12775C74E78E00
:101F3700048F05FF12774C900893ECF0A3EDF09017
:101F470000AEE05402601B9000A5E0A852B8001252
:101F5700D39553400DA204B3B35007E562C3949AD7
:101F67004002805FAE35AF369000A3E075F002A463
:101F7700FDACF0EF2DFDEE3CFC74022DFD50010C85
:101F8700E562BC003ED39D403A754401A23440331C
:101F97009000A4E075F05EA4FDACF07405FF127725
:101FA7004C8C5C8D5D124CCC900891E0FEA3E0FF59
:101FB7009000A4E02FFF50010E900891EEF0A3EFE0
:101FC700F0D234E562A835B8000495365002C23421
:101FD700856236753500E54470030220E6900101FD
:101FE700E0C3954450030220D8900111E0C3940246
:101FF7004003022082E56875F00A84FF7E009005A1
:1020070089120048E0F55B755A00AE5AAF5B900045
:10201700A4E012775C74648E048F05FF12774C8CF2
:102027005C8D5D900101E004C395448C068D071219
:10203700775C900101E08E048F05FF12774C8C5C72
:102047008D5D900891E0FEA3E0FFEF2DFDEE3CFCD7
:10205700900891ECF0A3EDF09000EFE0B4021A9035
:102067000893E0FEA3E0FFAA5CAB5DEF2BFBEE3A23
:10207700FA900893EAF0A3EBF08056900101E00490
:10208700C39544854CF0A4FFAEF0900101E08E04A7
:102097008F05FF12774C8C5C8D5D900891E0FEA355
:1020A700E0FFEF2DFDEE3CFC900891ECF0A3EDF086
:1020B7009000EFE0B4021A900893E0FEA3E0FFAAB5
:1020C7005CAB5DEF2BFBEE3AFA900893EAF0A3EBDB
:1020D700F00544900101E0C3954450037544009016
:1020E70000AEE05401601B9000A2E0A852B80012B5
:1020F700D39553400DA204B3B35007E560C394CC06
:10210700400280609000A0E075F003A4FFAEF0E508
:10211700412FFF50010E74032FFF50010EE560BEE3
:102127000042D39F403E754501A23440379000A13D
:10213700E075F05EA4FFAEF074058E048F05FF1204
:10214700774C8C5C8D5D124CCC900891E0FEA3E03F
:10215700FF9000A1E02FFF50010E900891EEF0A331
:10216700EFF0D234E560C395415002C23485604137
:10217700E5457003022280900102E0C395455003B4
:10218700022272900111E0C39402400302221CE56F
:102197006875F00A84FF7E00900589120048E0F513
:1021A7005B755A00AE5AAF5B9000A1E012775C7482
:1021B700648E048F05FF12774C8C5C8D5D90010255
:1021C700E004C395458C068D0712775C900102E009
:1021D7008E048F05FF12774C8C5C8D5D900891E023
:1021E700FEA3E0FFEF2DFDEE3CFC900891ECF0A381
:1021F700EDF09000EFE0B4021A900893E0FEA3E040
:10220700FFAA5CAB5DEF2BFBEE3AFA900893EAF07E
:10221700A3EBF08056900102E004C39545854DF08D
:10222700A4FFAEF0900102E08E048F05FF12774CF9
:102237008C5C8D5D900891E0FEA3E0FFEF2DFDEE35
:102247003CFC900891ECF0A3EDF09000EFE0B402B5
:102257001A900893E0FEA3E0FFAA5CAB5DEF2BFBAF
:10226700EE3AFA900893EAF0A3EBF00545900102E5
:10227700E0C395455003754500900891E0FEA3E043
:10228700FF9000B3E0BE00039F500D9000B3E090B5
:102297000891F8E4F0E8A3F09000EFE0B4021290A0
:1022A7000893E0FEA3E0FF9000B3E0BE00059F4067
:1022B70002800D9000B3E0900893F8E4F0E8A3F0F3
:1022C700229000EFE0B401028003022416A204B3B7
:1022D70050030223FD9000BAE0B4017A900891E020
:1022E700FEA3E0FFAC52AD53120003743C8E048F83
:1022F70005FF12774C9000CAE0BC00159D40129074
:102307000891E0FEA3E0FF9000CCE0BE00039F50E1
:1023170002D203900891E0FEA3E0FFAC52AD531246
:102327000003743C8E048F05FF12774C9000CAE0BF
:10233700C3940ABC001AD39D4016900891E0FEA3EF
:10234700E0FF9000CCE0C39405BE0004D39F500289
:102357008002C203807A900891E0FEA3E0FFAC52AE
:10236700AD5312000374788E048F05FF12774C90DB
:1023770000CAE0BC00159D4012900891E0FEA3E062
:10238700FF9000CCE0BE00039F5004D20380419031
:102397000891E0FEA3E0FFAC52AD5312000374783E
:1023A7008E048F05FF12774C9000CAE0C3940ABCD5
:1023B700001AD39D4016900891E0FEA3E0FF90001D
:1023C700CCE0C39405BE0004D39F50028002C20331
:1023D700A203B34021900891E0FEA3E0FF9000CB59
:1023E700E012775C74648E048F05FF12774C9008B7
:1023F70091ECF0A3EDF0A203B3400CA238400674B1
:1024070024900054F0D238A2034002C2388002C29E
:102417000390004FE06006A204B3B3400280199016
:102427000891E0FEA3E0FF90004FE02FFF50010E60
:10243700900891EEF0A3EFF0A201B34006A202B319
:10244700B3500990001AE4F0A3F0802D900891E0B2
:10245700FEA3E0FF7400D39F74019E401190089182
:10246700E0F8A3E090001AC8F0A3C8F0800B74FF4F
:1024770090001AF8E4F0E8A3F09000D1E0C39404C8
:10248700400C9008F3E0C3940240030225709000CB
:10249700BAE0B40147900891E0FEA3E0FF745E1232
:1024A700775C74058E048F05FF12774C900891ECCA
:1024B700F0A3EDF09000EFE0B4021F900893E0FE68
:1024C700A3E0FF745E12775C74058E048F05FF121C
:1024D700774C900893ECF0A3EDF08045900891E0DD
:1024E700FEA3E0FF745E12775C740A8E048F05FF0B
:1024F70012774C900891ECF0A3EDF09000EFE0B468
:10250700021F900893E0FEA3E0FF745E12775C74ED
:102517000A8E048F05FF12774C900893ECF0A3ED19
:10252700F0900891E0FEA3E0FF7402BE000CD39F79
:102537004008752A02752900800A900891E0F5295C
:10254700A3E0F52A900893E0FEA3E0FF7402BE0023
:102557000CD39F4008752E02752D00800A900893B2
:10256700E0F52DA3E0F52E8046900891E0FEA3E06C
:10257700FF7401BE000CD39F4008752A017529001E
:10258700800A900891E0F529A3E0F52A900893E0E6
:10259700FEA3E0FF7401BE000CD39F4008752E0117
:1025A700752D00800A900893E0F52DA3E0F52E9095
:1025B7000018E529F0A3E52AF0A23BB34009C201C0
:1025C70090001AE4F0A3F022900053E090038912E0
:1025D700778DE0F542754364900053E0FE9000C5A7
:1025E700E0D39E4037E56075F00884FF7E008F38A2
:1025F700E56075F00884ADF07C008D3B754008758B
:102607005A03755B96E538C3941F500512118880ED
:102617000690043EE0F5388538438035E56075F06F
:102627000884FF7E008F38E56075F00884ADF07C84
:10263700008D3B754008755A03755BB6E538C39442
:102647001F5005121188800690045EE0F538853822
:1026570043229000FBE0F53D754011755A04755B08
:1026670000AE52AF53E53D75F00FA4FDACF0EDD3CE
:102677009FEC9E4021E53D8E048F05FF12774CEDC0
:1026870075F010A4FFAEF0E56075F01184FD7C00D5
:10269700ED2FF53E800EE56075F01184FF7E00EFAB
:1026A70024F0F53E853E38E56075F01184AFF07E85
:1026B700008F3B12118885383FAE52AF539000FB15
:1026C700E075F00FA4FDACF0EDD39FEC9E402875AC
:1026D7005A04755B10853E38121188853F39853855
:1026E7003AAE52AF53E53D8E048F05FF1277778DD3
:1026F7003B853D3C121202853842754364229000A7
:10270700FBE0F53D754011755A04755B00AE52AF9D
:1027170053E53D75F00FA4FDACF0EDD39FEC9E4063
:1027270021E53D8E048F05FF12774CED75F010A45F
:10273700FFAEF0E56275F01184FD7C00ED2FF53EEC
:10274700800EE56275F01184FF7E00EF24F0F53E00
:10275700853E38E56275F01184AFF07E008F3B123D
:10276700118885383FAE52AF539000FBE075F00FEC
:10277700A4FDACF0EDD39FEC9E4028755A04755B21
:1027870010853E38121188853F3985383AAE52AFE9
:1027970053E53D8E048F05FF1277778D3B853D3CD2
:1027A7001212028538427543649000F6E0B404794A
:1027B700900053E0FE9000C5E0D39E4037E560757A
:1027C700F00884FF7E008F38E56075F00884ADF06F
:1027D7007C008D3B754008755A03755B96E538C3D9
:1027E700941F5005121188800690043EE0F5388545
:1027F70038438035E56075F00884FF7E008F38E543
:102807006075F00884ADF07C008D3B754008755A03
:1028170003755BB6E538C3941F500512118880060F
:1028270090045EE0F5388538432290008FE0B401CC
:102837003BE56875F00A84FF7E008F38E56875F020
:102847000A84ADF07C008D3B75400A755A05755BAF
:1028570012E538C39411500512118880069005AC13
:10286700E0F538E5432538C39464F543900090E0DC
:10287700B4013BE56975F00A84FF7E008F38E5698E
:1028870075F00A84ADF07C008D3B75400A755A05DA
:10289700755B7EE538C39411500512118880069048
:1028A7000618E0F538E5432538C39464F543E54257
:1028B7002543F537900097E0B402109008EBE02528
:1028C70037FE9000EBE0F4042EF5379000EEE0D3EE
:1028D70094014040E56CC394E7501D74E7C3956CC1
:1028E700FE9008EDE08E00F5F0E884FF7E008F385B
:1028F700E5372538F537801CE56CC394E7FE90086B
:10290700EDE08E00F5F0E884FF7E008F38E537C3F1
:102917009538F537A2044006E5422464F537E537D4
:10292700D394644009E537C39464F537800375375A
:10293700009000C7E0C3953750069000C7E0F53711
:1029470022D201900077E0A852B800049553503E78
:10295700900077E0A852B800049553500375370FDD
:10296700900077E004A852B80004955350037537D8
:1029770007900077E02402A852B80004955350024C
:10298700C201900077E060067409900054F0C233EA
:102997007E017F009000CDE012775C9000DCE08E36
:1029A700048F05FF12774CE560BC000CD39D4008EF
:1029B700D23B740A900054F090008FE0B401099064
:1029C70000CEE0C39568400280159000E0E0A85271
:1029D700B8000495535002C201740B900054F09054
:1029E700008FE0B40107E568C394644002801D903E
:1029F7000126E0600D900126E0A852B80006955325
:102A070040028008C201740B900054F0A2014003F9
:102A1700753700C23A90010FE0B40114900110E03D
:102A2700A852B8000495535007E560C3956140026A
:102A3700802A9000B8E0D3941D400B9000B8E0C303
:102A4700941EF5378003753700A237400874159038
:102A57000054F0D23AD237D235022B42C235C237B0
:102A6700900097E0B40306A22DB3B34003022B42B4
:102A77009008EFE0C39405A852B800049553500698
:102A87009008F6E06002801F9000B8E0D3941D40E4
:102A97000B9000B8E0C3941EF537800375370074B8
:102AA7000C900054F0D23A9008EFE0A852B8000416
:102AB700955350069008F6E07002801F9000B8E02A
:102AC700D3941D400B9000B8E0C3941EF5378003E4
:102AD700753700740C900054F0D23A9008EFE0A8D4
:102AE70052B80004955350319000D6E0B40228D272
:102AF700339008F5E0FE9008F6E0D39E5006900864
:102B0700F6E0700280099008F5E4F0C23380069081
:102B170008F5E004F08002C2019008EFE02405A860
:102B270052B80004955350139000D6E0B4020A90AF
:102B370008F6E07002D2338002C201A232B3402706
:102B47009000B8E0D3941D400B9000B8E0C3941EEA
:102B5700F5378003753700A236400674109000548D
:102B6700F0D236D23A8002C23685376D9000B8E08F
:102B7700D3941D4018900086E02537FE900053E05F
:102B870075F01E84FC7F00EE2CF5378029A23AB33E
:102B97004008900086E0F537801C900088E02537D4
:102BA700FE900086E02EFE900053E075F01E84FC38
:102BB7007F00EE2CF537A23BB34005D233756D008D
:102BC70022900053E075F00584FF7E008F38900057
:102BD70053E075F00584ADF07C008D3B75400575BD
:102BE7005A03755BD69000DAE01475F00584FF7E12
:102BF70000E538BE00039F5005121188800BE538A9
:102C070090045F12778DE0F538E5389008EEF09084
:102C170008EEE0FE9000C9E0C39E50089000C9E0AE
:102C27009008EEF09000B8E0D3941D401E9008EE97
:102C3700E0FE900086E02EFE900053E075F01E84C3
:102C4700FC7F00EE2C9008EEF08031A23AB3400AE8
:102C5700900086E09008EEF080229008EEE0FE906B
:102C67000088E02EFE900086E02EFE900053E0756F
:102C7700F01E84FC7F00EE2C9008EEF02290008F6F
:102C8700E0B40136E56875F00A84FF7E0090058997
:102C9700120048E0F547E547D394644010E547C381
:102CA700946475F00F84FF7E008F4780037547009B
:102CB7009000ACE02547F54780069000ACE0F5476B
:102CC70022E56875F00A84FF7E00900589120048A6
:102CD700E0C394694007E568D3946440559000F6D3
:102CE700E0C39403502690088BE0FEA3E0FF740432
:102CF700120039E56012775C740F8E048F05FF129E
:102D0700774C900889ECF0A3EDF0802490088BE0D5
:102D1700FEA3E0FF7404120039E56212775C740FBA
:102D27008E048F05FF12774C900889ECF0A3EDF025
:102D3700800F90088BE0F8A3E0900889C8F0A3C83B
:102D4700F0A204401A90088BE0FEA3E0FF74031280
:102D5700775C7401120039900889EEF0A3EFF090C8
:102D6700009FE0B40262E56BC3944175F00584FFF0
:102D77007E008F38E56B75F00584ADF07C008D3BE8
:102D8700754005755A06755B14E538C394175005E9
:102D970012118880069006B0E0F538900889E0FEA9
:102DA700A3E0FF740A8E048F05FF12774CE5388C79
:102DB700068D0712775C740A8E048F05FF12774C15
:102DC700900889ECF0A3EDF0900889E0FEA3E0FFFE
:102DD70090088FE0FCA3E0FDEDD39FEC9E400F90A1
:102DE700088FE0F8A3E0900889C8F0A3C8F022E5AF
:102DF7000875F004A4FFAEF09006CC120048E090EE
:102E07003C4BF8282873804C85537480479000DC2E
:102E1700E08560F0A4FFAEF074081200398F74806B
:102E270033856274802E856874802985697480244F
:102E3700856A74801F856B74801A856C748015850C
:102E470067748010856674800B856D7480069000AA
:042E57001BE0F57413
:103C4B00022E0D022E0F022E14022E28022E2D02F2
:103C5B002E32022E37022E3C022E41022E46022E0F
:073C6B004B022E50022E5502
:102E5B00E50875F004A4FFAEF09006CD120048E52E
:102E6B000875F004A4FFAEF0E0FC9006CE1200480B
:102E7B00ECFEE0FFEEC39F4003022F63E50875F005
:102E8B0004A4FFAEF09006CC120048E0B40441E578
:102E9B000875F004A4FFAEF09006CE120048E0C314
:102EAB009574500AE508F50CD3923C123DAEE5083B
:102EBB0075F004A4FFAEF09006CD120048E0D39558
:102ECB0074400AE508F50CC3923C123DAE022F612B
:102EDB00E50875F004A4FFAEF09006CD120048E0B3
:102EEB00C395745015E50875F004A4FFAEF0900679
:102EFB00CE120048E0D395745002800AE508F50C19
:102F0B00D3923C123DAEE50875F004A4FFAEF090F1
:102F1B0006CD120048E0D395745015E50875F00402
:102F2B00A4FFAEF09006CE120048E0C39574500A91
:102F3B00E508F50CC3923C123DAE9006D4E0B4010B
:102F4B00099000E8E0D395625002800A7402F50CF8
:102F5B00C3923C123DAE806AE50875F004A4FFAE47
:102F6B00F09006CD120048E0D395744015E5087536
:102F7B00F004A4FFAEF09006CE120048E0C39574A7
:102F8B004002800AE508F50CC3923C123DAEE50801
:102F9B0075F004A4FFAEF09006CD120048E0C39587
:102FAB00744015E50875F004A4FFAEF09006CE1240
:102FBB000048E0D39574400AE508F50CD3923C1217
:102FCB003DAE22AE2FAF3074C9BE000CD39F40086C
:102FDB00782F1277AF0230E8753001752F00AE52A3
:102FEB00AF53E547BE000DD39F40099000BEE0D321
:102FFB00954840028023754800E547C39553F57407
:10300B009000C1E0D395464008E5462574F546800F
:10301B00069000C1E0F5468002054890009AE0D387
:10302B009562401CE560C395614015AE52AF53E508
:10303B0047BE00039F50099000BFE0D39549400263
:10304B00806E9008F0E0A852B800049553500375B9
:10305B004B009008F0E0A852B8000BD395534006F4
:10306B00E5539008F0F0E54B7041E553C39547F5F8
:10307B0074E574D3940540037574059000C0E0C3E8
:10308B0095465007E574C3954640028009E546C353
:10309B009574F54680069000C0E0F5469000C0E0C0
:1030AB00D3954640069000C0E0F546754900800276
:1030BB000549E54B701690009AE0C39562500DE5FB
:1030CB00472405A852B8000695534002800F900084
:1030DB00ADE0F546754B0174789008F0F022AE2FF9
:1030EB00AF3074E9D39F74039E4008782F1277AFEB
:1030FB0002328F753001752F00754632A22E402A91
:10310B007546199000ADE075F002A4FFAEF0E548EE
:10311B00BE0006D39F4002D22E0548754B03747830
:10312B009008F0F0754A00023276AE52AF53E54785
:10313B006F4E7003023276E547BE000DD39F4009F8
:10314B009000BEE0D395484002800F754800E54BD8
:10315B00C394035003754619800DE547C39553F58A
:10316B0074E5482574F54890009AE0D39562400EBB
:10317B009008F0E0A852B80007D395534002800C9A
:10318B00054A9000ADE0B54A03754B00E54BB4031F
:10319B0006A204B3B34002800A054AE54AB43C03D5
:1031AB00754B02E54BB402299008F0E0A852B80029
:1031BB000ED395534009E5539008F0F0754A0090F3
:1031CB00009AE0C395625009754A0074789008F034
:1031DB00F0E54B705A90009AE0D39562401CE56085
:1031EB00C395614015AE52AF53E547BE00039F50E8
:1031FB00099000BFE0D395494002800875490075DE
:10320B00464B8028E553C39547F574E574D3940575
:10321B00400375740590009AE0D395624008E54928
:10322B002574F5498006E5492406F549754A00E5FC
:10323B004B701690009AE0C39562500DE54724053C
:10324B00A852B80006955340028003754B01E54B1D
:10325B00B40118754619054A9000ADE0B54A0675DC
:10326B004B02754A0074789008F0F0A202B3400349
:10327B00754632E54675F00AA4FFAEF0900895EE60
:10328B00F0A3EFF022E570903C72F8282873023C13
:10329B000B900092E070030235BA9000C8E0B401C5
:1032AB00028003023450900051E0655F6009E553E2
:1032BB004552600302344D7E017F00E5BE12775C00
:1032CB00E5BD2FFF50010E8E5A8F5B9000C6E0B408
:1032DB00461B740E12775C900076E08E048F05FF10
:1032EB0012774C900899ECF0A3EDF0801DAE5AAF1D
:1032FB005B741012775C900076E08E048F05FF12E2
:10330B00774C900899ECF0A3EDF0E56C600FE56C51
:10331B00C394FE50089000EEE0640260028064905B
:10332B0000DCE0B40B1F900899E0FEA3E0FF74E70C
:10333B0012775CE56C8E048F05FF12774C90089921
:10334B00ECF0A3EDF09000DCE0D3940B4008900080
:10335B00C4E064046002802B900899E0FEA3E0FFB8
:10336B0090089DE0FCA3E0FDEFD39DEE9C400D1279
:10337B0077A7900899EEF0A3EFF08007900899E4F7
:10338B00F0A3F0900899E0FEA3E0FFEFD39400EEDA
:10339B0094014008D23B7426900054F0A23BB3B387
:1033AB00502C7E057F009000DCE08E048F05FF1211
:1033BB00774C900899E0FEA3E0FFEFC39DEE9C4095
:1033CB000FAC52AD53740FBC0004D39D500280025E
:1033DB00C23B900092E0B4022790089BE0FEA3E072
:1033EB00FF900899E0FCA3E0FDEF2DFDEE3CFC7493
:1033FB00018C068D07120039900899EEF0A3EFF0BF
:10340B00900899E0FEA3E0FF90089BE0FCA3E0FD91
:10341B00EDD39FEC9E4004D2318002B231900899DB
:10342B00E0F8A3E090089BC8F0A3C8F09000C4E0BC
:10343B0064016006A231B3B34002800690089AE0A3
:10344B00F5600235B8D2317E017F00E5BE12775CA4
:10345B00E5BD2FFF50010E8E5A8F5B9000C6E0B476
:10346B00461B740E12775C900076E08E048F05FF7E
:10347B0012774C900899ECF0A3EDF0801DAE5AAF8B
:10348B005B741012775C900076E08E048F05FF1250
:10349B00774C900899ECF0A3EDF0E56C600FE56CC0
:1034AB00C394FE50089000EEE064026002806490CA
:1034BB0000DCE0B40B1F900899E0FEA3E0FF74E77B
:1034CB0012775CE56C8E048F05FF12774C90089990
:1034DB00ECF0A3EDF09000DCE0D3940B40089000EF
:1034EB00C4E064046002802B900899E0FEA3E0FF27
:1034FB0090089DE0FCA3E0FDEFD39DEE9C400D12E8
:10350B0077A7900899EEF0A3EFF08007900899E465
:10351B00F0A3F0900899E0FEA3E0FFEFD39400EE48
:10352B0094014008D23B7426900054F0A23BB3B3F5
:10353B00502C7E057F009000DCE08E048F05FF127F
:10354B00774C900899E0FEA3E0FFEFC39DEE9C4003
:10355B000FAC52AD53740FBC0004D39D50028002CC
:10356B00C23B900092E0B4022790089BE0FEA3E0E0
:10357B00FF900899E0FCA3E0FDEF2DFDEE3CFC7401
:10358B00018C068D07120039900899EEF0A3EFF02D
:10359B00900899E0F8A3E090089BC8F0A3C8F090BE
:1035AB0000C4E06401600690089AE0F56080037542
:1035BB00600090008EE0700675700302329075BB50
:1035CB0018023C0B023C0B90008EE0700302374359
:1035DB007E017F00E5BE12775CE5BD2FFF50010E2B
:1035EB008E5A8F5B9000D4E0B4010F7E0F7FFFAC3F
:1035FB005AAD5B1277A78E5A8F5B9000F9E0B4023D
:10360B0045AE5AAF5B900024E0FCA3E0FDEDD39FE9
:10361B00EC9E400A900024E55AF0A3E55BF0AE5A0D
:10362B00AF5B900026E0FCA3E0FDEFD39DEE9C404A
:10363B000A900026E55AF0A3E55BF0AE5AAF5B7437
:10364B00041200398F629000F9E0704CAE5AAF5BF8
:10365B00900024E0FCA3E0FDEFD39DEE9C4009120B
:10366B0077A78E5A8F5B8006755B00755A00AE5A32
:10367B00AF5B741012775C9000F8E08E048F05FF3F
:10368B0012774C8C5A8D5B74FFBC0009D39D40059F
:10369B00855B6280037562FE9000C4E0B40102801A
:1036AB0003023741A204B3B3500E900098E0A85226
:1036BB00B80005D39553500280719000D5E0856218
:1036CB00F0A4FFAEF074648E048F05FF12774C8C60
:1036DB005A8D5BE56C6016E56CC394FE500F900041
:1036EB00EEE0B402089000DCE0640B60028017AEE1
:1036FB005AAF5B74E712775CE56C8E048F05FF1293
:10370B00774C8C5A8D5BAE5AAF5B900899E0FCA35B
:10371B00E0FDEDD39FEC9E4005855B60800BA231F5
:10372B00B3400690089AE0F560800BA231B34006D7
:10373B0090089AE0F5608003756200900091E0704C
:10374B000675700502329075BB19023C0B023C0BDF
:10375B00900091E070030237FBE55FD3955E400369
:10376B000237F9900022E0FEA3E0FFE56612779F97
:10377B00900022EEF0A3EFF07E017F00E5BE127702
:10378B005CE5BD2FFF50010E8E5A8F5B9000FEE063
:10379B007013740A12775C74518E048F05FF1277C5
:1037AB004C8D668019AE5AAF5B740A12775C8F042E
:1037BB008E057E017F95CDCCCD12764A8F66E56660
:1037CB00D394644003756664900022E0FEA3E0FF8F
:1037DB00E5662FFF50010E900022EEF0A3EFF09064
:1037EB000095E0048E048F05FF12774C8D668003E5
:1037FB007566329000E1E0700675700702329075C5
:10380B00BB13023C0B023C0B9000E1E0604A7E01D3
:10381B007F00E5BE12775CE5BD2FFF50010E8E5A7F
:10382B008F5B74041200398F679000E3E08567F0BB
:10383B00A4FDACF07464FF12774C8D679000E2E04E
:10384B008567F0A4FFAEF074FF8E048F05FF12772F
:10385B004CED900075F0800375670090008FE07061
:10386B000675700902329075BB17023C0B023C0BBC
:10387B0090008FE0B40102800302390F7E017F00BC
:10388B00E5BE12775CE5BD2FFF50010E8E5A8F5BA4
:10389B009008F1E060199008F1E01490713C12006F
:1038AB008CE493FC740193FDEDC39FEC9E4002806E
:1038BB00069008F1E014F09008F1E0C394B3501DAA
:1038CB00AE5AAF5B9008F1E00490713C12008CE4AF
:1038DB0093FC740193FDEFC39DEE9C400280069018
:1038EB0008F1E004F09008F1E0FE9000B5E08E00E6
:1038FB0088F0A4FFAEF074648E048F05FF12774C32
:10390B008D688003756800900090E0700675700BF1
:10391B0002329075BB16023C0B023C0B900090E000
:10392B00B4010280030239BB7E017F00E5BE127732
:10393B005CE5BD2FFF50010E8E5A8F5B9008F2E0B5
:10394B0060199008F2E0149072A612008CE493FCBC
:10395B00740193FDEDC39FEC9E400280069008F22C
:10396B00E014F09008F2E0C394B3501DAE5AAF5B75
:10397B009008F2E0049072A612008CE493FC7401A0
:10398B0093FDEFC39DEE9C400280069008F2E0048D
:10399B00F09008F2E0FE9000BBE08E0088F0A4FFF0
:1039AB00AEF074648E048F05FF12774C8D69800323
:1039BB0075690075BB1F023C0B023C0B7E017F003F
:1039CB00E5BE12775CE5BD2FFF50010E8E5A8F5B63
:1039DB00740912775C74E68E048F05FF12774C8D99
:1039EB006B900097E0700675700F02329075BB15E7
:1039FB00023C0B023C0B900097E07003023B527EA3
:103A0B00017F00E5BE12775CE5BD2FFF50010E8EE6
:103A1B005A8F5B74041200398F6A900097E0B401DF
:103A2B00159000EBE0856AF0A4FFAEF0740712006E
:103A3B0039EF9008ECF0900097E0B402159000EB92
:103A4B00E0856AF0A4FFAEF07407120039EF90081E
:103A5B00EBF0900097E0B403028003023B3590003B
:103A6B00D8E07052E56AC39419500FD22D9000B76D
:103A7B00E09008EFF09008F4E4F0E56AD39464402A
:103A8B0004A22D4002802D9008F4E004F09008F47D
:103A9B00E0FE90012AE0B5060B9008EFE004F090F1
:103AAB0008F4E4F09008EFE06496600690012AE0D9
:103ABB007002C22D80639000B7E070349000EBE091
:103ACB00856AF0A4FFAEF074FF8E048F05FF1277AA
:103ADB004CED9008EFF0AE52AF53741EBE0006D300
:103AEB009F4002D22DE562D394E54002C22D80297E
:103AFB00E56AC3940A500DAE52AF53741EBE000458
:103B0B00D39F50028002D22DE562D394E54002C2CE
:103B1B002D9000B7E09008EFF09008EFE0C394050C
:103B2B00500674059008EFF0C232900097E0B40491
:103B3B0014E56AC394195002D232E56AD394324029
:103B4B0002C232C22D8003756A009000EEE070064F
:103B5B0075701102329075BB14023C0B023C0B903A
:103B6B0000EEE07003023BF87E017F00E5BE1277AA
:103B7B005CE5BD2FFF50010E8E5A8F5B900113E059
:103B8B007025EFD39421EE940E4005756CFF8015D4
:103B9B00AE5AAF5B741012775C74E38E048F05FF23
:103BAB0012774C8D6C8027AE5AAF5BEFD39449EEF6
:103BBB0094064005756CFF8015AE5AAF5B741012FE
:103BCB00775C74638E048F05FF12774C8D6CE56CFC
:103BDB0075F00BA4FFAEF09000DCE08E048F05FFB8
:103BEB0012774C90089DECF0A3EDF08003756C0000
:103BFB00900092E0600575BB1A800375BB188000BE
:103C720002329902329C0235CF0235D20237580203
:103C8200375B02381002381302387802387B023967
:103C9200240239270239C40239C70239FE023A0125
:093CA200023B67023B6A023C0B85
:103C0B00E57075F00284AFF07E00EF4E7002D2ECDF
:033C1B000570220F
:09778D002582F5825002058322D9
:0F008C0025E050020583258250020583F582226C
:10772B00EF2F500205832582F582E5833E2EF583EC
:01773B00222B
:10779F00CFC39FFF50011E22C3EF9DFFEE9CFE2221
:0877AF000806B60002180622CC
:0D776A00A3E004F07006127783E004F02223
:0E003900048007C3CE13CECF13CFD5E0F6223E
:10764A00BC000FBE0008ED8FF084FFADF022E4FE0F
:10765A00FF22BE000DEF60FE54F0606F20E70302C8
:10766A007700EAC0E0EBC0E078017A0075F001EE3D
:10767A0020E710EF25E0FFEE33FE0AC5F023C5F040
:10768A0030E7F0EA5407F9096A7A007B00600108DA
:10769A00C3EC9E40167004ED9F4010ED9FFDEC9EDA
:1076AA00FCE5F0CA4ACA03F5F08005E5F003F5F0F7
:1076BA00C3EE13FEEF13FFD9D77908CACBCAD8D0C5
:1076CA00EAFEEBFFD0E0FBD0E0FA22EC8FF084FC7C
:1076DA00ED54F045F0C48FF084FEEDC454F045F04B
:1076EA00C48FF084FDEEC4FE54F02DFFEE540F3C1F
:1076FA00FEADF07C0022790078008FF0EC7E082045
:10770A00E70DC3CD33CD33C933C9C833C8DEF084DE
:10771A0049F9E5F08FF0BE00E6FD7C00E9FFE8FEDE
:01772A00223C
:0E775C00F88FF0A4FFE5F0CE88F0A42EFE22F8
:10000300EF8DF0A4F9A8F0EF8CF0A428F8EE8DF0B2
:06001300A428FEE9FF2213
:10773C00600D782B027746007830D8FED5E0F82221
:10774C00EEC0E07E0012764AEFFDEEFCD0E0FE22A9
:0C777700EEC0E07E0012764AD0E0FE2258
:03001B0002001EC2
:0300530002005652
:03009B00020071EF
:03000000027796EE
:0977960075817675D000024E8F5A
:0B004800E5822FF582E5833EF5832260
:0A7783000582D582021583158222CB
:10001E00C0E0C0F0C083C082C0D075D000124D9237
:0B002E00D0D0D082D083D0F0D0E032E0
:10005600C0E0C0F0C083C082C0D075D000124D95FC
:10006600D0D0D082D083D0F0D0E032C0E0C0F0C093
:1000760083C082C0D075D000124DF3D0D0D082D0CC
:0600860083D0F0D0E0324F
:00000001FF
